:100000000C94B7080C94DF080C94DF080C94DF08FC
:100010000C94DF080C94DF080C94DF080C94DF08C4
:100020000C94DF080C94DF080C94DF080C94DF08B4
:100030000C94DF080C94DF080C94DF080C94DF08A4
:100040000C94DF080C94DF080C9481560C94DF08A4
:100050000C94D0590C94175A0C94DF080C94DF08B8
:100060000C94DF080C94DF080C94D2540C94DF0835
:10007000485454502F312E3020323030204F4B0D09
:100080000A436F6E74656E742D547970653A2074EE
:100090006578742F68746D6C0D0A507261676D61BC
:1000A0003A206E6F2D63616368650D0A4163636575
:1000B00073732D436F6E74726F6C2D416C6C6F7720
:1000C0002D4F726967696E3A202A0D0A0D0A0048A1
:1000D0005454502F312E3020323030204F4B0D0AE7
:1000E000436F6E74656E742D547970653A2061703B
:1000F000706C69636174696F6E2F6A736F6E0D0A3D
:10010000436F6E6E6E656374696F6E3A20636C6FD9
:1001100073650D0A4163636573732D436F6E74726B
:100120006F6C2D416C6C6F772D4F726967696E3AF9
:10013000202A0D0A0D0A003C6D657461206E616D08
:10014000653D76696577706F727420636F6E746554
:100150006E743D2277696474683D363430223E0DFA
:100160000A00485454502F312E302034303120555D
:100170006E617574686F72697A65640D0A436F6E9B
:1001800074656E742D547970653A20746578742F97
:1001900068746D6C0D0A0D0A3C68313E34303120B4
:1001A000556E617574686F72697A65643C2F683149
:1001B0003E0077696E646F772E6C6F636174696F50
:1001C0006E3D222F223B3C2F7363726970743E0A8E
:1001D000006376007670006D7000647000637000DC
:1001E000677000766F00636F00736E007073007647
:1001F00073006373007672006372006A6F006A6E48
:10020000006A70006A63006A7300737500637500AA
:1002100074730024460024440024460024463C6DA8
:1002200065746120687474702D65717569763D22FE
:10023000726566726573682220636F6E74656E7492
:100240003D22313B2075726C3D2F223E005D2C22F9
:100250006E73746174696F6E73223A24447D002C4E
:10026000002444007B22736E223A5B002446002463
:10027000463C7363726970743E616C6572742822C7
:100280004F7074696F6E732076616C75657320733F
:10029000617665642E22293B24460024463C736324
:1002A000726970743E616C65727428224E657720A5
:1002B00070617373776F726473206D757374206DE2
:1002C000617463682122293B77696E646F772E6CB5
:1002D0006F636174696F6E3D222F766F223B3C2FF6
:1002E0007363726970743E0A0024463C73637269DA
:1002F00070743E616C65727428224E65772070615F
:100300007373776F7264207365742E22293B2446C1
:100310000024463C7363726970743E616C6572744C
:10032000282256616C756573206F7574206F662086
:10033000626F756E642122293B77696E646F772E38
:100340006C6F636174696F6E3D222F766F223B3C48
:100350002F7363726970743E0A0024463C736372A3
:100360006970743E616C657274282253637269709F
:10037000742075726C2073617665642E22293B248B
:10038000460024463C7363726970743E24460052F2
:1003900065626F6F74696E672E2E2E0024463C6D69
:1003A00065746120687474702D65717569763D227D
:1003B000726566726573682220636F6E74656E7411
:1003C0003D2224443B2075726C3D2F223E003C733D
:1003D0006372697074207372633D2224452F7669BD
:1003E00065776F702E6A73223E3C2F73637269705B
:1003F000743E0A003C2F7363726970743E0A0030C9
:100400005D3B766172206E6F7074733D24442C6C7A
:100410006F633D222445222C646576743D244C2C68
:10042000747A3D24443B00222446222C24442C246C
:10043000442C24442C003C7363726970743E7661D2
:1004400072206F7074733D5B0024462446007D006B
:100450002C00222446223A2444007B002446003CFF
:10046000736372697074207372633D2224452F6830
:100470006F6D652E6A73223E3C2F736372697074D0
:100480003E0A000A766172206C72756E3D5B2444F0
:100490002C24442C24442C244C5D3C2F736372691F
:1004A00070743E0A005B302C305D5D3B0A766172F1
:1004B00020656E3D24442C72643D24442C72733DAF
:1004C00024442C6D6D3D24442C726473743D244C83
:1004D0002C6D61733D24442C7572733D24442C773C
:1004E0006C3D24442C697061733D24442C6C6F6313
:1004F0003D222445223B005B24442C244C5D2C00EF
:10050000305D3B7661722070733D5B0024442C00AB
:10051000766172206E6272643D24442C747A3D24AC
:10052000442C73626974733D5B007661722076655A
:10053000723D24442C646576743D244C3B0A0024AF
:100540004624463C7363726970743E003C6469766D
:100550002069643D226F7574707574223E64756DF8
:100560006D793C2F6469763E003C2F73637269702D
:10057000743E0073657454696D656F757428226EDE
:100580006577414A4158436F6D6D616E6428276AF3
:1005900063272C2066756E632C2074727565292282
:1005A0002C31303030293B0066756E6374696F6E94
:1005B0002066756E632864617461297B76617220A0
:1005C0006A643D4A534F4E2E7061727365286461B0
:1005D0007461293B24242822236F7574707574225A
:1005E000292E746578742864617465737472286A3E
:1005F000645B2264657674225D2A313030302929AB
:100600003B7D0066756E6374696F6E20696E6974F8
:1006100028297B66756E6328227B5C22646576746C
:100620005C223A307D22293B7D00242428696E69B2
:1006300074293B003C7363726970743E0D0A003C80
:10064000736372697074207372633D22687474708E
:100650003A2F2F3139322E3136382E312E31303378
:100660002F6D6368702E6A73223E3C2F736372692C
:1006700070743E0D0A003C7363726970742073726B
:10068000633D2268747470733A2F2F6A71756572B6
:10069000796A732E676F6F676C65636F64652E632D
:1006A0006F6D2F66696C65732F6A71756572792D30
:1006B000312E332E322E6D696E2E6A73223E3C2F00
:1006C0007363726970743E0D0A0024462446005B11
:1006D000302C305D5D2C226C72756E223A5B2444A6
:1006E0002C24442C24442C244C5D7D005B24442C7D
:1006F000244C5D2C00305D2C227073223A5B002468
:10070000442C007B2264657674223A244C2C226EA1
:10071000627264223A24442C22656E223A24442CCC
:10072000227264223A24442C227273223A24442CEA
:10073000226D6D223A24442C2272647374223A246E
:100740004C2C226C6F63223A222445222C227362A5
:10075000697473223A5B0024460077696E646F7790
:100760002E6C6F636174696F6E3D222F7670223B31
:100770003C2F7363726970743E0A00616C65727419
:10078000282250726F6772616D202444206D6F645F
:10079000696669656422293B00616C657274282270
:1007A0004E65772070726F6772616D206164646559
:1007B000642E22293B0024463C7363726970743EA8
:1007C000003C736372697074207372633D22244528
:1007D0002F706C6F7470726F672E6A73223E3C2F9D
:1007E0007363726970743E0A00305D3B0024442CD0
:1007F00000766172206D61736F703D5B007661728F
:10080000207365713D24442C6D61733D24442C7725
:100810006C3D24442C7364743D24442C6D746F6EC1
:100820003D24442C6D746F66663D24442C646576CB
:100830006461793D24442C6465766D696E3D244481
:100840002C64643D24442C6D6D3D24442C79793D09
:1008500024443B0024463C7363726970743E002458
:10086000463C7363726970743E77696E646F772E6D
:100870006C6F636174696F6E3D222F7670223B3C12
:100880002F7363726970743E0A003C2F7363726940
:1008900070743E0A3C736372697074207372633DB6
:1008A0002224452F6D6F6470726F672E6A73223E2B
:1008B0003C2F7363726970743E0A005D3B002C2408
:1008C00044007661722070726F673D5B24442C2473
:1008D000442C24442C24442C24442C24442C2444F0
:1008E00000766172206E626F617264733D24442CE5
:1008F0007069643D24442C697061733D24443B005D
:10090000244624463C7363726970743E003C7363F2
:1009100072697074207372633D2224452F76696575
:100920007770726F672E6A73223E3C2F7363726911
:1009300070743E0A00244624463C736372697074E6
:100940003E0024463C7363726970743E2446003C4A
:10095000736372697074207372633D2224452F762D
:10096000696577726F2E6A73223E3C2F73637269DA
:1009700070743E0A00305D3B3C2F73637269707483
:100980003E0A0024442C00766172206E626F617210
:1009900064733D24442C6D61733D24442C69706163
:1009A000733D24442C6475723D5B00244624463C10
:1009B0007363726970743E005D7D005D005D2C00A4
:1009C0002C2444005B24442C24442C24442C244414
:1009D0002C24442C24442C2444007B226E70726FFF
:1009E0006773223A24442C226E626F617264732210
:1009F0003A24442C226D6E70223A24442C227064D6
:100A0000223A5B002446003C6872202F3E3C666F11
:100A1000726D206E616D653D6F6620616374696FF4
:100A20006E3D6375206D6574686F643D6765743EE7
:100A30003C703E3C623E4A617661736372697074D9
:100A40002055524C3A3C2F623E203C696E707574C2
:100A500020747970653D746578742073697A653D9A
:100A60003332206D61786C656E6774683D31323762
:100A70002076616C75653D22244522206E616D658E
:100A80003D6A73703E3C2F703E3C703E536574204F
:100A900055524C207768657265204A6176617363B0
:100AA0007269707473206172652073746F7265640B
:100AB0002E2044656661756C742069732024533C54
:100AC0006272202F3E4966206C6F63616C206F6EEE
:100AD0002075534420636172642C20757365202E49
:100AE0002028692E652E20646F74293C2F703E3CAF
:100AF000703E3C623E50617373776F72643A3C2F74
:100B0000623E3C696E70757420747970653D7061E9
:100B10007373776F72642073697A653D3130206E2C
:100B2000616D653D70773E3C696E707574207479B7
:100B300070653D7375626D69743E3C2F703E3C6814
:100B400072202F3E3C2F666F726D3E002446003CA3
:100B50002F7363726970743E0A005D3B002C24445D
:100B60000070645B24445D3D5B24442C24442C24AD
:100B7000442C24442C24442C24442C24440076610A
:100B800072206E70726F67733D24442C6E626F61C9
:100B90007264733D24442C697061733D24442C6D50
:100BA0006E703D24442C70643D5B5D3B0024463CEC
:100BB0007363726970743E616C6572742822436855
:100BC000616E6765732073617665642E22293B240C
:100BD000460027275D3B00272453272C00766172AF
:100BE00020736E616D65733D5B00305D3B3C2F7320
:100BF00063726970743E0A3C736372697074207327
:100C000072633D2224452F76696577736E2E6A7371
:100C1000223E3C2F7363726970743E0A0024442C98
:100C200000305D3B7661722069723D5B0024442C8C
:100C300000766172206D61736F703D5B007661724A
:100C4000206E626F617264733D24442C6D61786C18
:100C5000656E3D24442C6D61733D24442C697061A4
:100C6000733D24443B0024463C7363726970743EB8
:100C7000005D2C226D61786C656E223A24447D0003
:100C80002C002444005D2C2269676E6F72655F72D0
:100C900061696E223A5B002C002444005D2C226DB9
:100CA00061736F70223A5B002C0022245322007B78
:100CB00022736E616D6573223A5B002446004E54C8
:100CC000502053796E63696E672E2E2E00436F6E2F
:100CD0006E656374696E672E2E2E004465746563BD
:100CE00074696E67207553442E2E2E000001080093
:100CF0000604000145000082000040002000504F23
:100D0000535420244620485454502F312E300D0A7D
:100D1000486F73743A2024460D0A244624534163D5
:100D2000636570743A202A2F2A0D0A436F6E74652A
:100D30006E742D4C656E6774683A2024440D0A4326
:100D40006F6E74656E742D547970653A20617070A1
:100D50006C69636174696F6E2F782D7777772D6674
:100D60006F726D2D75726C656E636F6465640D0ACC
:100D70000D0A245300474554202446245320485448
:100D800054502F312E300D0A486F73743A20244688
:100D90000D0A24460D0A0D0A004163636570743A1A
:100DA00020746578742F68746D6C00E30004FA0099
:100DB000010000000166777600747A006E7470009E
:100DC0006468637000697031006970320069703363
:100DD00000697034006777310067773200677733D6
:100DE000006777340068703000687031006172000D
:100DF0006578740073657100736474006D617300CD
:100E00006D746F6E006D746F66007572730072732F
:100E10006F00776C007374740069706173006465AF
:100E200076696400636F6E006C69740064696D00BC
:100E30006E747031006E747032006E747033006EB8
:100E4000747034007265736574004669726D776101
:100E50007265207665722E0054696D65207A6F6E1A
:100E6000653A004E54502073796E633F00557365A8
:100E700020444843503F005374617469632E697085
:100E8000313A005374617469632E6970323A0053C9
:100E900074617469632E6970333A005374617469C4
:100EA000632E6970343A00476174657761792E6901
:100EB00070313A00476174657761792E6970323A12
:100EC00000476174657761792E6970333A00476134
:100ED00074657761792E6970343A00485454502013
:100EE000706F72743A00004175746F207265636FA1
:100EF0006E6E6563743F0023206F66206578702EE8
:100F000020626F6172643A0053657175656E746931
:100F1000616C206D6F64653F0053746174696F6E1E
:100F20002064656C61793A004D6173746572207359
:100F3000746174696F6E3A004D617374657220203C
:100F40006F6E2061646A2E3A004D61737465722081
:100F50006F66662061646A2E3A005573652072617F
:100F6000696E2073656E736F723A004E6F726D61B9
:100F70006C6C79206F70656E3F0025205761746539
:100F8000722074696D653A0053656C66746573749C
:100F90002074696D653A0049676E6F7265207061F3
:100FA0007373776F72643F004465766963652049A7
:100FB000443A004C434420436F6E74726173743A38
:100FC000004C4344204261636B6C696768743A006B
:100FD0004C43442044696D6D696E673A004E54502D
:100FE000207365727665722E6970313A004E5450E6
:100FF000207365727665722E6970323A004E5450D5
:10100000207365727665722E6970333A004E5450C3
:10101000207365727665722E6970343A005265737A
:10102000657420616C6C3F004D6F6E0054756500F7
:101030005765640054687500467269005361740016
:1010400053756E00206D696E002073656300250086
:101050004E6F00596573002B002B0020474D540044
:101060003030003A002D002B000020202020002DE1
:1010700044697361626C6564212D003A0045004D3E
:10108000433A003A002E002D0020002020003A00B4
:10109000200042333A686F6C6420746F207361766D
:1010A000650042333A73656C2042312F42323A6315
:1010B0006867003D3D536574204F7074696F6E73AF
:1010C0003D3D00506C6561736520576169742E2E3B
:1010D0002E00526573657474696E672045455052E1
:1010E0004F4D0000002100240027002A00000022AC
:1010F00000250028002B00000020002300260029E6
:1011000000020202020202020204040404040404B3
:1011100004030303030303030301010101010101AC
:101120000101020408102040800102040810204040
:101130008001020408102040808040201008040232
:10114000010000000102000000000000000403078D
:101150000600000000000000000000000000000089
:1011600000004D0BAA39104765486E53F75A1124F9
:101170001FBECFEFD0E1DEBFCDBF13E0A0E0B1E0F6
:10118000E4EFF9EB02C005900D92AE39B107D9F743
:101190001DE0AEE9B3E001C01D92AF3EB107E1F73B
:1011A00011E1CEE6D1E104C02297FE010E94BD5CB0
:1011B000C236D107C9F70E94475B0C94F85C0C94C7
:1011C0000000FC0188279927E89421912032E9F357
:1011D000293010F02E30C8F32B3241F02D3239F483
:1011E000689404C00E941B0A820F911D2191205314
:1011F0002A30C0F31EF4909581959F4F08951F9358
:10120000FC0199278827BC01E89411911032E9F379
:10121000193010F01E30C8F31B3251F01D3249F462
:10122000689406C00E94060A610F711D811D911D00
:10123000119110531A30B0F33EF49095809570954B
:1012400061957F4F8F4F9F4F1F910895FB01DC01E8
:1012500002C005900D9241505040D8F70895FB010F
:10126000DC0104C08D910190801921F4415050405F
:10127000C8F7881B990B0895DC0101C06D9341509C
:101280005040E0F70895FB01DC018D910190801939
:101290000110D9F3990B0895FB01DC0101900D9227
:1012A0000020E1F70895FB01DC014150504030F08F
:1012B0008D910190801919F40020B9F7881B990BC2
:1012C0000895A0E0B0E0E7E6F9E00C94CB5C7C0187
:1012D000EB018A01690109C0CE012196F601099549
:1012E000F70181937F010150104001151105A1F70D
:1012F000CDB7DEB7E8E00C94E75CBF92CF92DF9207
:10130000EF92FF920F931F937B018C01FB010995D4
:10131000B82EC8010196F7010995C82EC80102969A
:10132000F7010995D82EC8010396F7010995982F62
:101330006B2D7C2D8D2D1F910F91FF90EF90DF90E5
:10134000CF90BF900895A0E0B0E0E9EAF9E00C94F6
:10135000CB5CEC017B018A01690109C0CE012196B9
:10136000F70161917F01F6010995015010400115C7
:101370001105A1F7CDB7DEB7E8E00C94E75CBF92AA
:10138000CF92DF92EF92FF920F931F93D52EC62E2E
:10139000B72E79018C01642FF9010995C8010196D6
:1013A0006D2DF7010995C80102966C2DF70109957D
:1013B000C80103966B2DF70109951F910F91FF90BE
:1013C000EF90DF90CF90BF900895FB019F01E894CC
:1013D0004230C4F04532B4F44A3029F497FB1EF48D
:1013E000909581959F4F642F77270E94725C805D56
:1013F0008A330CF0895D8193CB010097A1F716F435
:101400005DE251931082C9010C94480A592F482F6C
:10141000372F262F660F771F881F991F660F771F9C
:10142000881F991F620F731F841F951F660F771FF8
:10143000881F991F08957AE0979F902D879F802D90
:10144000910D11240895FA01CF93FF93EF93223069
:10145000CCF02532BCF4C22F2C2F3327442755273C
:10146000FF93EF930E94995CEF91FF91605D6A3367
:101470000CF0695D6193B901CA0160507040804011
:10148000904051F710828F919F91CF910C94480A10
:10149000DC01FC01672F71917723E1F7329704C0DB
:1014A0007C916D9370836291AE17BF07C8F3089566
:1014B0009C01F999FECF32BD21BDF89A80B50895FF
:1014C0009C01F999FECF1FBA32BD21BD60BD0FB698
:1014D000F894FA9AF99A0FBE0895FC01A681B78193
:1014E0006D93B783A68381E090E00895CF92DF9259
:1014F000EF92FF920F931F93CF93DF937B018C01A9
:101500000894E11CF11C011D111DC090520C4423D4
:1015100061F430914F0C3695369536953170AAE2CC
:10152000B8E0CAE6D7E0DD2471C090914F0C9695E3
:10153000969596959170CAE2D8E06AE677E0EC2D30
:10154000F0E0EE0FFF1FEE0FFF1FEC0FFD1F25C099
:10155000288139814A815B81211531054105510579
:10156000C9F0DB01ED92FD920D931C931397D80106
:10157000C701820F931FA41FB51F88839983AA8375
:10158000BB8320919E027C018D01E20EF11C011DA6
:10159000111D91E024966C5F7F4FCE17DF07C1F6D7
:1015A0009170990F990F990F80914F0C877F892B1C
:1015B00037C04D915D916D917C9113974115510507
:1015C0006105710501F1ED2DE695E695E695F0E0F2
:1015D000ED5AF34F808190E02D2D277002C0959534
:1015E00087952A95E2F780FD0EC0E882F9820A838A
:1015F0001B834E0D5F1D601F711F4D935D936D9397
:101600007C93139731E0D39414962496DC1488F2DB
:101610003170330F330F330F80914F0C877F832B43
:1016200080934F0CDF91CF911F910F91FF90EF901E
:10163000DF90CF900895AAEEB8E080E090E0FC0142
:10164000E659F84F1082118212821382FC01E65D86
:10165000F74F10821182128213821D920496803CF1
:10166000910569F7F999FECF8CE694E092BD81BDB2
:10167000F89A80B580936107109262071092630711
:101680001092650710926407109266071092670720
:1016900010926807109269070895109258071092E7
:1016A000570782E393E09093560780935507089578
:1016B0009F92AF92BF92CF92DF92EF92FF920F93E1
:1016C0001F93CF93DF93EC01962E81EC99E0BE013E
:1016D0000E94FD3C882309F458C081EC99E0BE01CA
:1016E00041E00E94E33DAA24BB24650181EC99E01E
:1016F0000E94DE39EC01A2E0BAE026E330E040E0EF
:1017000050E0A20EB31EC41ED51EF501E056FC4FDC
:101710002AEC3FEF4FEF5FEFA20EB31EC41ED51EA3
:101720008601750107C00894E11CF11C011D111D03
:101730008D918193C7018A199B098C179D079CF392
:1017400030E0E31632E0F30630E0030730E0130741
:1017500048F0C70160E144E00E94C630AA24BB24DF
:1017600065010AC041E0941629F4C70161E144E033
:101770000E94C63057016801C050D24009F4B6CF6C
:1017800081EC99E00E94A33981E0DF91CF911F9114
:101790000F91FF90EF90DF90CF90BF90AF909F9010
:1017A0000895AF92BF92DF92EF92FF920F931F9333
:1017B000CF93DF9300D000D000D0EDB7FEB73196C5
:1017C00005E517E0ADB7BEB712961C930E931197BF
:1017D0008CE692E0938382838FEC90E09583848300
:1017E0000E94E9350F900F90EDB7FEB71283018389
:1017F00084E692E0948383830E94E935FF240F906E
:101800000F900F900F90D02EE12E21E6A22E22E015
:10181000B22ECFE5D2E04FC00F2D10E000D000D0A7
:1018200000D0ADB7BEB71196EDB7FEB7D182E28258
:101830001396BC92AE921297F80193E0F595E79556
:101840009A95E1F7ED5AF34F808190E09801277067
:10185000307002C0959587952A95E2F78170907057
:1018600015969C938E9314970E94E9358091520CA3
:1018700090E001972DB73EB72A5F3F4F0FB6F8941F
:101880003EBF0FBE2DBF08171907A1F000D000D032
:10189000ADB7BEB71196DC9211971296EC921297E3
:1018A0001496DC93CE9313970E94E9350F900F9016
:1018B0000F900F90F3942091520CF21608F4ACCFD5
:1018C00000D000D000D0EDB7FEB7319685E597E0A7
:1018D000ADB7BEB712969C938E9311978DE492E0AC
:1018E00093838283248315820E94E935EDB7FEB786
:1018F00036960FB6F894FEBF0FBEEDBF81E0DF91C4
:10190000CF911F910F91FF90EF90DF90BF90AF901C
:101910000895AF92BF92CF92DF92EF92FF920F9312
:101920001F93CF93DF9300D000D000D0EDB7FEB768
:10193000319605E517E0ADB7BEB712961C930E932E
:1019400011978CE594E0938382838FEC90E09583EC
:1019500084830E94E9350F900F90EDB7FEB7128394
:1019600001838AE594E0948383830E94E935C7E28A
:10197000D2E0FF240F900F900F900F90E02E012FD8
:1019800042E5A42E44E0B42E30E5C32E34E0D32E3D
:101990002C813D818881F4E1FF1619F490E0CC9709
:1019A00001C090E04DB75EB7485050400FB6F89474
:1019B0005EBF0FBE4DBFEDB7FEB73196ADB7BEB738
:1019C0001196EC92119712960C93B382A2823583F2
:1019D0002483978386830E94E935EDB7FEB7389656
:1019E0000FB6F894FEBF0FBEEDBFF2E2FF16A1F0F6
:1019F00000D000D0ADB7BEB71196EC9211971296F9
:101A00000C9312971496DC92CE9213970E94E935AC
:101A10000F900F900F900F90F3942796B3E2FB1660
:101A200009F0B6CF00D000D085E597E0EDB7FEB75E
:101A3000928381838EE494E0948383830E94E935CA
:101A40000F900F900F900F9081E0DF91CF911F9139
:101A50000F91FF90EF90DF90CF90BF90AF900895DF
:101A60000F931F938DB79EB708970FB6F8949EBF3C
:101A70000FBE8DBFEDB7FEB7319605E517E0ADB7E8
:101A8000BEB712961C930E9311978AEC96E093833F
:101A9000828380E790E09583848387E391E0978356
:101AA00086830E94E9350F900F900F900F90EDB74D
:101AB000FEB71283018386E796E0948383830E94B6
:101AC000E935ADB7BEB712961C930E9311978FE30D
:101AD00096E014969C938E9313970E94E935EDB788
:101AE000FEB71283018384E396E0948383830E948C
:101AF000E935ADB7BEB712961C930E9311978AE2E3
:101B000096E014969C938E9313970E94E935EDB757
:101B1000FEB71283018383E096E0948383830E945F
:101B2000E935ADB7BEB712961C930E93119788EAAC
:101B300095E014969C938E9313970E94E935EDB728
:101B4000FEB71283018383E795E0948383830E9429
:101B5000E935ADB7BEB712961C930E93119789E67F
:101B600095E014969C938E9313970E94E935EDB7F8
:101B7000FEB7128301838CE495E0948383830E94F3
:101B8000E9350F900F900F900F9081E01F910F910A
:101B900008950F931F9300D000D000D0EDB7FEB78B
:101BA000319605E517E0ADB7BEB712961C930E93BC
:101BB00011978CE49BE09383828380E790E0958388
:101BC00084830E94E93500D0EDB7FEB73196ADB7FA
:101BD000BEB712961C930E93119787E09AE09383F9
:101BE000828380E890E09583848380E091E097830E
:101BF00086830E94E9358DB79EB708960FB6F89494
:101C00009EBF0FBE8DBF81E01F910F910895CF92AF
:101C1000DF92EF92FF920F931F93DF93CF9300D049
:101C200000D0CDB7DEB70E94C9567B018C016E0192
:101C30000894C11CD11C0E94E02D0E94F432C60100
:101C40006091AB010E94EC2F8823E1F0E980FA80DB
:101C50000B811C8180EC98EDA4E5BCE7E80EF91E31
:101C60000A1F1B1F60912E0270E080E090E024E8C4
:101C700033E040E050E00E94475CE60EF71E081F8C
:101C8000191F0EC00E94C9566E197F09800B910B57
:101C9000685E73408040904070F2EE24FF2487011C
:101CA000B701C8010F900F900F900F90CF91DF9167
:101CB0001F910F91FF90EF90DF90CF900895EF92DA
:101CC000FF921F93DF93CF9300D000D0CDB7DEB744
:101CD0008091F9028983809100038A8380910703B0
:101CE0008B8380910E038C8310E07E010894E11CAD
:101CF000F11C6091AB016F5F6093AB01C7010E9463
:101D000056326AEF70E080E090E00E94D7560E9461
:101D1000070E9B01AC01611571058105910519F450
:101D20001F5F143131F7B901CA010F900F900F9066
:101D30000F90CF91DF911F91FF90EF900895CF9377
:101D4000DF939C0110922407FC01A081B181C0E0C7
:101D5000D0E00FC09C919D3231F09B3221F0892F51
:101D600080538A3068F4FE01EC5DF84F9083219631
:101D70001196F901808191810A96A817B90750F34D
:101D8000CC5DD84F18821196F901B183A08384E20B
:101D900097E00E94E108DF91CF910895BF92CF9222
:101DA000DF92EF92FF920F931F93CF93DF932DB7A4
:101DB0003EB7285030400FB6F8943EBF0FBE2DBF3F
:101DC000EDB7FEB7319605E517E0ADB7BEB7129691
:101DD0001C930E93119789E494E09383828380E7A8
:101DE00090E09583848387E391E0978386830E94C4
:101DF000E9350F900F900F900F90EDB7FEB712835B
:101E0000018386E394E0948383830E94E93557E25B
:101E1000E52E52E0F52EDD24C0E0D0E00F900F90CB
:101E20000F900F90B02EC12E07E214E05C2F6D2FA3
:101E3000D70116968C91169781FF33C014962D9179
:101E40003C91159711964C9111978C91C43119F4CE
:101E500090E0CC9701C090E0EDB7FEB73C970FB68D
:101E6000F894FEBF0FBEEDBF3196ADB7BEB7119669
:101E7000BC9211971296CC921383028335832483EC
:101E80004683178291878087528763870E94E9354E
:101E9000D394EDB7FEB73C960FB6F894FEBF0FBED5
:101EA000EDBF219627E030E0E20EF31EC332D105EC
:101EB00009F0BCCF0E94FD44ADB7BEB71E970FB668
:101EC000F894BEBF0FBEADBFEDB7FEB7319605E5C6
:101ED00017E012961C930E9311972FEF33E0338384
:101EE0002283D482158220E630E037832683608700
:101EF00071878287938780912E02848715860E943E
:101F0000E935EDB7FEB73A960FB6F894FEBF0FBEAF
:101F1000EDBF1283018384EF93E0948383830E9457
:101F2000E93500D0EDB7FEB73196ADB7BEB7129622
:101F30001C930E9311978EEC93E09383828380E839
:101F400090E0958384830E94E935EDB7FEB736961D
:101F50000FB6F894FEBF0FBEEDBF81E0DF91CF91C9
:101F60001F910F91FF90EF90DF90CF90BF90089559
:101F70004F925F926F927F928F929F92AF92BF9299
:101F8000CF92DF92EF92FF920F931F93DF93CF9345
:101F90000F92CDB7DEB70E94FD445B016C0100D00B
:101FA00000D000D0EDB7FEB7319605E517E0ADB72C
:101FB000BEB712961C930E93119787E597E0938313
:101FC00082838FEC90E0958384830E94E935EDB79E
:101FD000FEB772970FB6F894FEBF0FBEEDBF3196F5
:101FE000ADB7BEB712961C930E93119783E097E09E
:101FF00093838283A482B582C682D7828091510C5A
:102000008087118680914F0C817082871386809122
:102010004F0C869581708487158680914F0C86952C
:10202000869581708687178680914F0C8295817086
:10203000808B118A8091650C9091660CA091670C41
:10204000B091680C828B938BA48BB58B80E690E06B
:10205000978B868B0E94E93590E0EDB7FEB77896B6
:102060000FB6F894FEBF0FBEEDBF78010FEF16E07C
:1020700023C000D000D000D0EDB7FEB73196ADB789
:10208000BEB71196EC9211971296FC9213830283BD
:10209000A92FB0E0AD5AB34F8C91848315829983F8
:1020A0000E94E93599819F5FEDB7FEB736960FB66E
:1020B000F894FEBF0FBEEDBF8091510CA5E56A2ECE
:1020C000A7E07A2E9817A8F200D000D0ADB7BEB71F
:1020D00012967C926E92119785EF96E014969C93DF
:1020E0008E9313970E94E93599240F900F900F90CB
:1020F0000F90C301762C892EFCEE4F2EF6E05F2E5A
:1021000066C0A92DB0E0FD01E651F74F608166235E
:10211000A9F1CD01880F991F880F991FFC01E6597D
:10212000F84FE080F18002811381FC01E65DF74FFA
:10213000AE14BF04C006D10648F02081318142812F
:1021400053812A193B094C095D0908C0208131815E
:10215000428153812E193F09400B510BAA0FBB1F1F
:10216000AA0FBB1FA65DB74F8D919D910D90BC919D
:10217000A02D8E5F9F4FAF4FBF4F21F420E030E086
:1021800040E050E08DB79EB70A970FB6F8949EBF17
:102190000FBE8DBFEDB7FEB73196ADB7BEB7119686
:1021A0007C92119712968C9253824282648315829C
:1021B00026833783408751870E94E9359394EDB792
:1021C000FEB73A960FB6F894FEBF0FBEEDBF8091F2
:1021D000520C981608F495CF2DB73EB72E503040CC
:1021E0000FB6F8943EBF0FBE2DBFEDB7FEB73196C8
:1021F00085E597E0ADB7BEB712969C938E93119785
:102200008FEC96E0938382838091620784831582AA
:102210008091630786831782809164079091650798
:10222000918780878091660790916707A0916807E2
:10223000B091690782879387A487B5870E94E935A3
:10224000EDB7FEB73E960FB6F894FEBF0FBEEDBFDA
:1022500081E00F90CF91DF911F910F91FF90EF9050
:10226000DF90CF90BF90AF909F908F907F906F90B6
:102270005F904F900895BF92CF92DF92EF92FF92BE
:102280000F931F936C01FC01B080E1800E94FD441C
:1022900020E831E541E050E00E94995C8B2D8F777A
:1022A000280F311D411D511DFF2400E010E0CA011F
:1022B000B901A80197010E94995CF0E8BF22B62AF3
:1022C000F601B0821F910F91FF90EF90DF90CF90B9
:1022D000BF9008956F927F928F929F92AF92BF921C
:1022E000CF92DF92EF92FF920F931F934C01FC016C
:1022F000708061800E94FD44A62CBB24CC24DD2488
:10230000BFE7EB2EE720FF24E60CF11C0027F7FCCB
:102310000095102F20E831E541E050E00E94995CE3
:10232000CA01B901A60195010E94995CE61AF70A53
:10233000080B190BC801B701A60195010E94995C11
:10234000F0E87F22762AF40170821F910F91FF90AE
:10235000EF90DF90CF90BF90AF909F908F907F9045
:102360006F900895EF92FF921F93CF93DF93182FF2
:102370007B010E94FD449B01AC01C12FD0E02F5F87
:102380003F4F4F4F5F4FCE01880F991F880F991F06
:10239000FC01E659F84F2083318342835383FC01CB
:1023A000E65DF74FE114F10449F48EEF9FEFAFEFD4
:1023B000BFEF80839183A283B3830DC0C701AA2797
:1023C00097FDA095BA2F280F391F4A1F5B1F208346
:1023D000318342835383C651D74F83E688838091EC
:1023E0004F0C886080934F0CDF91CF911F91FF902D
:1023F000EF900895AF92BF92CF92DF92EF92FF924B
:102400000F931F93CF93DF938C010E5F1F4F20E03C
:1024100030E006C0F901ED5DF84F90830F5F1F4F6C
:10242000E22FD8019C91892F80538A3028F42F5FA6
:102430003F4F2530310571F7F0E0EC5DF84F108229
:1024400084E297E00E94E108EC0197FDD4C08091FE
:10245000520C90E08C179D070CF4CDC0F8018081E0
:102460008D3309F057C0209709F4C5C080914F0CF7
:1024700084FFC1C02197C80101962181203379F4DE
:102480000E94FD44EC2FF0E0EE0FFF1FEE0FFF1F48
:10249000E65DF74F608371838283938319C0213394
:1024A00009F0A9C064E277E040E32BE231E00E944A
:1024B0004750882319F460E070E007C084E297E099
:1024C0000E94E108BC0197FD96C08C2F0E94B211BA
:1024D00000D000D000D0EDB7FEB7319685E597E08B
:1024E000ADB7BEB712969C938E9311978CE192E094
:1024F0009383828380E790E0958384830E94E9350B
:1025000081E0EDB7FEB736960FB6F894FEBF0FBE6A
:10251000EDBF72C000D000D000D0EDB7FEB731964D
:1025200085E597E0ADB7BEB712969C938E93119751
:1025300089E192E09383828380E790E095838483AE
:102540000E94E935EDB7FEB736960FB6F894FEBF98
:102550000FBEEDBF209721F48091520C90E003C094
:102560008C2F9C2F9150C0E0D0E0E92EFF24082F43
:1025700010E065E5A62E67E0B62E56E1C52E52E0C6
:10258000D52E31C000D000D000D0ADB7BEB7119667
:10259000EDB7FEB7B282A1821396DC92CE9212976B
:1025A000F90143E0F595E7954A95E1F7ED5AF34FC8
:1025B000808190E02770307002C0959587952A95AC
:1025C000E2F78170907015969C938E9314970E94F9
:1025D000E93521962DB73EB72A5F3F4F0FB6F894E5
:1025E0003EBF0FBE2DBF9E012E0D3F1D2017310790
:1025F0004CF281E001C080E0DF91CF911F910F91FB
:10260000FF90EF90DF90CF90BF90AF900895BF9272
:10261000CF92DF92EF92FF920F931F93CF93DF93AE
:1026200000D000D005E517E0ADB7BEB712961C93F9
:102630000E9311978DED9BE014969C938E931397B8
:102640000E94E935FF240F900F900F900F90B02E4D
:10265000E12EB4E2CB2EB7E0DB2E07ED1BE021C06C
:102660008F2D64E277E00E94304700D000D000D088
:10267000EDB7FEB73196ADB7BEB71196BC921197C4
:102680001296EC9213830283D582C4820E94E935AC
:10269000F394EDB7FEB736960FB6F894FEBF0FBEB3
:1026A000EDBF8091520CC5E5D7E0F816C8F200D016
:1026B00000D0ADB7BEB71296DC93CE93119782EDE2
:1026C0009BE014969C938E9313970E94E9350F908C
:1026D0000F900F900F908E819F812C813D81821BE6
:1026E000930B60E140E00E94C630DF91CF911F91D3
:1026F0000F91FF90EF90DF90CF90BF9008954F9291
:102700005F926F927F928F929F92AF92BF92CF9281
:10271000DF92EF92FF920F931F93DF93CF930F926D
:10272000CDB7DEB70E94FD445B016C012DB73EB70B
:10273000285030400FB6F8943EBF0FBE2DBFEDB706
:10274000FEB7319605E517E0ADB7BEB712961C93FC
:102750000E9311978FE395E09383828380E790E057
:102760009583848387E391E0978386830E94E9358C
:10277000EDB7FEB738960FB6F894FEBF0FBEEDBFAB
:102780000E940713109258071092570786ED93E0A6
:1027900090935A078093590790935C0780935B0747
:1027A0002DB73EB72A5030400FB6F8943EBF0FBE4B
:1027B0002DBFEDB7FEB73196ADB7BEB712961C93DD
:1027C0000E9311978AE295E0938382838DEC90E0DB
:1027D00095838483A682B782C086D1860E94E9351C
:1027E0000F900F90EDB7FEB73196ADB7BEB712960A
:1027F0001C930E93119780E195E0938382838091DF
:10280000510C8483158280912E02868317820E9448
:10281000E93590E0EDB7FEB738960FB6F894FEBFF5
:102820000FBEEDBF78010CE015E023C000D000D052
:1028300000D0EDB7FEB73196ADB7BEB71196EC92AA
:1028400011971296FC9213830283A92FB0E0AD5A20
:10285000B34F8C918483158299830E94E9359981C5
:102860009F5FEDB7FEB736960FB6F894FEBF0FBE6A
:10287000EDBF8091510C25E5622E27E0722E98174E
:10288000A8F200D000D0ADB7BEB712967C926E927F
:10289000119780E095E014969C938E9313970E9475
:1028A000E93599240F900F900F900F90C301762C6B
:1028B000892E87EF482E84E0582E66C0A92DB0E0FF
:1028C000FD01E651F74F60816623A9F1CD01880F24
:1028D000991F880F991FFC01E659F84FE080F1809D
:1028E00002811381FC01E65DF74FAE14BF04C00600
:1028F000D10648F020813181428153812A193B0958
:102900004C095D0908C020813181428153812E1913
:102910003F09400B510BAA0FBB1FAA0FBB1FA65D9F
:10292000B74F8D919D910D90BC91A02D8E5F9F4FC3
:10293000AF4FBF4F21F420E030E040E050E08DB7D2
:102940009EB70A970FB6F8949EBF0FBE8DBFEDB726
:10295000FEB73196ADB7BEB711967C92119712961D
:102960008C92538242826483158226833783408708
:1029700051870E94E9359394EDB7FEB73A960FB6AA
:10298000F894FEBF0FBEEDBF8091520C981608F46C
:1029900095CF2DB73EB72A5130400FB6F8943EBFC1
:1029A0000FBE2DBFEDB7FEB7319605E517E0ADB709
:1029B000BEB712961C930E93119785EA94E0938309
:1029C000828380914F0C81708483158280914F0C9B
:1029D000869581708683178280914F0C86958695A7
:1029E00081708087118680914F0C829581708287DB
:1029F00013868091650C9091660CA091670CB09144
:102A0000680C84879587A687B7878091A502808BFD
:102A1000118A8091BA02828B138A8091C802848BBA
:102A2000158A8091D602868B178A80E690E0918F76
:102A3000808F0E94E935EDB7FEB73C960FB6F8944B
:102A4000FEBF0FBEEDBF3196ADB7BEB712961C9359
:102A50000E93119783E894E09383828380916207B9
:102A6000848315828091630786831782809164072F
:102A7000909165079187808780916607909167079D
:102A8000A0916807B091690782879387A487B5876B
:102A90000E94E935EDB7FEB738960FB6F894FEBF41
:102AA0000FBEEDBF3196ADB7BEB712961C930E9315
:102AB00011978FE594E09383828380E890E095837B
:102AC00084830E94E935EDB7FEB736960FB6F894C9
:102AD000FEBF0FBEEDBF81E00F90CF91DF911F9140
:102AE0000F91FF90EF90DF90CF90BF90AF909F90AD
:102AF0008F907F906F905F904F900895FF920F930B
:102B00001F93CF93DF938C010E945231109258078C
:102B10001092570786ED93E090935A0780935907D8
:102B200090935C0780935B07A8014B5F5F4FD801D0
:102B300015968C91803221F4CA010E947F136EC0D9
:102B4000CCEAD1E0A0E0B0E0682F772767FD709570
:102B5000FA2EE881F981849190E08617970709F0B1
:102B60006CC03196249130E0FA018181992787FD6C
:102B700090952817390709F060C0AA0FBB1FAA0F4C
:102B8000BB1FA255BE4FED91FC91CA010995882348
:102B900001F500D000D000D0EDB7FEB7319685E545
:102BA00097E0ADB7BEB712969C938E93119783E1D1
:102BB00092E09383828382E691E0958384830E94EE
:102BC000E935EDB7FEB736960FB6F894FEBF0FBEE7
:102BD000EDBFF5E1FF1611F580914F0C86FF1EC089
:102BE000402FE4E2F7E0C801DC0101C081939A2F95
:102BF000941B15968C911597803229F0119627E039
:102C0000E434F20799F7E92FF0E0EC5DF84F108219
:102C100084E297E061E00E94580B17C080915B0747
:102C200090915C072091590730915A07821B930BB2
:102C300061E140E00E94C63008C0F39411962496EA
:102C4000A531B10509F084CFC4CFDF91CF911F9199
:102C50000F91FF900895BF92CF92DF92EF92FF9273
:102C60000F931F93CF93DF932DB73EB7285030407B
:102C70000FB6F8943EBF0FBE2DBFEDB7FEB731962D
:102C800005E517E0ADB7BEB712961C930E931197EA
:102C90008BEA99E09383828380E790E09583848335
:102CA00087E391E0978386830E94E935EDB7FEB70D
:102CB00038960FB6F894FEBF0FBEEDBF0E94071303
:102CC000109258071092570786ED93E090935A0799
:102CD0008093590790935C0780935B072DB73EB7AD
:102CE0002A5030400FB6F8943EBF0FBE2DBFEDB74F
:102CF000FEB73196ADB7BEB712961C930E931197DF
:102D000087E899E0938382838091510C84831582B4
:102D10008091A502868317828091D60280871186D2
:102D20000E94E935DD24E12C44E0F42EEDB7FEB736
:102D30003A960FB6F894FEBF0FBEEDBFB02EC12E6F
:102D400003E819E033C0F999FECFF2BCE1BCF89A70
:102D500090B5F999FECF0894E11CF11CF2BCE1BCDE
:102D6000F89A80B5D92FC0E000D000D000D0EDB7E0
:102D7000FEB73196ADB7BEB71196BC9211971296B9
:102D8000CC92138302839E01280F311D3583248347
:102D90000E94E935D3940894E11CF11C8DB79EB7CD
:102DA00006960FB6F8949EBF0FBE8DBF8091520C51
:102DB000D81608F4C8CF00D000D005E517E0ADB7AD
:102DC000BEB712961C930E93119785E799E014965F
:102DD0009C938E9313970E94E93500D0EDB7FEB710
:102DE0003196ADB7BEB712961C930E9311978FE430
:102DF00099E09383828380E890E0958384830E94A6
:102E0000E935EDB7FEB736960FB6F894FEBF0FBEA4
:102E1000EDBF81E0DF91CF911F910F91FF90EF9077
:102E2000DF90CF90BF900895AF92BF92DF92EF9264
:102E3000FF920F931F93DF93CF930F92CDB7DEB71F
:102E400000D000D000D0EDB7FEB7319605E517E011
:102E5000ADB7BEB712961C930E93119786E69CE011
:102E60009383828380E790E0958384830E94E93591
:102E7000EDB7FEB736960FB6F894FEBF0FBEEDBFA6
:102E80000E940713109258071092570786ED93E09F
:102E900090935A078093590790935C0780935B0740
:102EA0002DB73EB72C5030400FB6F8943EBF0FBE42
:102EB0002DBFEDB7FEB73196ADB7BEB712961C93D6
:102EC0000E9311978DE39CE0938382838091510C44
:102ED0008483158280E190E0978386838091A502A8
:102EE000808711868091D602828713860E94E935F9
:102EF000EDB7FEB738960FB6F894FEBF0FBEEDBF24
:102F00001283018381E39CE0948383830E94E935EB
:102F100090E00F900F900F900F9078010DE21CE061
:102F200023C000D000D000D0EDB7FEB73196ADB7CA
:102F3000BEB71196EC9211971296FC9213830283FE
:102F4000A92FB0E0A75AB34F8C918483158299833F
:102F50000E94E93599819F5FEDB7FEB736960FB6AF
:102F6000F894FEBF0FBEEDBF8091510C75E5A72E02
:102F700077E0B72E9817A8F200D000D0ADB7BEB753
:102F80001296BC92AE92119781E29CE014969C93AB
:102F90008E9313970E94E93500E00F900F900F90E9
:102FA0000F90C501DA2C192F6DE1E62E6CE0F62E9C
:102FB00021C000D000D000D0EDB7FEB73196ADB73C
:102FC000BEB71196DC92119712961C93F382E2829F
:102FD000A02FB0E0A15AB34F8C91848315820E9438
:102FE000E9350F5FEDB7FEB736960FB6F894FEBF22
:102FF0000FBEEDBF8091510C55E5A52E57E0B52EC3
:103000000817B8F200D000D000D0EDB7FEB7319667
:10301000ADB7BEB71296BC92AE9211978AEE9BE006
:103020009383828380E890E0958384830E94E935CE
:10303000EDB7FEB736960FB6F894FEBF0FBEEDBFE4
:1030400081E00F90CF91DF911F910F91FF90EF9052
:10305000DF90BF90AF9008958F929F92AF92BF92F2
:10306000CF92DF92EF92FF920F931F93CF93DF9354
:1030700000D000D000D0EDB7FEB7319605E517E0DF
:10308000ADB7BEB712961C930E9311978BEB9CE0D5
:10309000938382838FEC90E0958384830E94E9354B
:1030A0000F900F90EDB7FEB7128301838FEA9CE07B
:1030B000948383830E94E935FF240F900F900F9033
:1030C0000F90E02E012F94E2C92E97E0D92E8AEAC4
:1030D000882E8CE0982E18EAA12E1CE0B12E3EC05E
:1030E0008F2D64E277E00E94304700D000D000D0FE
:1030F000EDB7FEB73196ADB7BEB71196EC9211970A
:1031000012960C9393828282D582C4820E94E93502
:103110002F2D30E08091520C90E00197EDB7FEB773
:1031200036960FB6F894FEBF0FBEEDBF28173907CD
:10313000A1F000D000D0ADB7BEB71196EC921197B8
:1031400012960C9312971496BC92AE9213970E940B
:10315000E9350F900F900F900F90F3948091520CDF
:10316000C5E5D7E0F81608F4BBCF00D000D0EDB726
:10317000FEB7D283C1838CE99CE0948383830E9451
:10318000E935FF240F900F900F900F90CE01DC2EA9
:10319000E92EB9E98B2EBCE09B2EA7E9AA2EACE064
:1031A000BA2E40C00F2D10E000D000D000D0ADB737
:1031B000BEB71196EDB7FEB7D182E28213969C920C
:1031C0008E921297F801E75AF34F808114968C93F0
:1031D000149715961C920E94E9358091510C90E04D
:1031E00001972DB73EB72A5F3F4F0FB6F8943EBF09
:1031F0000FBE2DBF08171907A1F000D000D0ADB742
:10320000BEB71196DC9211971296EC921297149613
:10321000BC92AE9213970E94E9350F900F900F90D9
:103220000F90F3948091510CC5E5D7E0F81608F49F
:10323000B9CF00D000D0EDB7FEB7D283C18385E807
:103240009CE0948383830E94E935FF240F900F90C4
:103250000F900F90CE01DC2EE92EF2E88F2EFCE0CD
:103260009F2EE0E8AE2EECE0BE2E40C00F2D10E009
:1032700000D000D000D0ADB7BEB71196EDB7FEB705
:10328000D182E28213969C928E921297F801E15AB3
:10329000F34F808114968C93149715961C920E947C
:1032A000E9358091510C90E001972DB73EB72A5F28
:1032B0003F4F0FB6F8943EBF0FBE2DBF081719073A
:1032C000A1F000D000D0ADB7BEB71196DC92119737
:1032D0001296EC9212971496BC92AE9213970E949B
:1032E000E9350F900F900F900F90F3948091510C4F
:1032F000C5E5D7E0F81608F4B9CF00D000D000D06B
:10330000EDB7FEB73196ADB7BEB71296DC93CE934C
:10331000119781E79CE09383828380E190E095831D
:1033200084830E94E935EDB7FEB736960FB6F89460
:10333000FEBF0FBEEDBF81E0DF91CF911F910F91D6
:10334000FF90EF90DF90CF90BF90AF909F908F90C5
:1033500008959C018091D602882311F081E00895A0
:10336000C90164E277E040E32DE231E00E9447507A
:10337000882331F084E297E00E944648811181E081
:1033800008954F925F926F927F928F929F92AF9229
:10339000BF92CF92DF92EF92FF920F931F93DF9332
:1033A000CF93CDB7DEB7E5970FB6F894DEBF0FBE6B
:1033B000CDBF33E0A32EB12CA80EB91EC5010E94CB
:1033C000A919882309F436C150902E024090350285
:1033D00007E212E0EE24CC24DD244E010894811C87
:1033E000911C22E0622E712C6C0E7D1E2C2D9D2DC9
:1033F000D80116968C91169781FF3BC011968C913F
:103400001197813009F41C92D401E6E3F3E085E0E2
:1034100001900D928150E1F7822FB3014AE050E014
:103420000E94E509C50164E277E040E394010E944F
:1034300047508823F1F0F801F180F1E0FF1619F40C
:10344000D801FC9216C084E297E00E94E1089C013A
:10345000B4E1CB1611F4245C3F4F37FD08C08F2D2B
:1034600090E0821793071CF0F801208302C0EE243D
:10347000E3940894C11CD11C095F1F4FF3E2CF16DF
:10348000D10409F0B3CFC50164E277E040E320E363
:1034900031E00E944750882351F084E297E00E9477
:1034A000935080E690E064E277E00E942148C501F5
:1034B00064E277E040E324E331E00E944750882350
:1034C000C1F084E297E00E94935084E297E00E946A
:1034D000FF08162F072FF82ED92E0E94D044809176
:1034E0004F0C85FF06C0612F702F8F2D9D2D0E94E0
:1034F000D046EE2089F000D000D000D0EDB7FEB766
:10350000319685E597E0ADB7BEB712969C938E9342
:10351000119781E193E0B5C00E94FD47C50164E2C7
:1035200077E040E328E331E00E944750882309F424
:1035300044C08E010A5F1F4FC501B80140E32CE370
:1035400031E00E944750882309F48BC084E297E061
:10355000B80140E150E00E945309009709F081C092
:1035600080E490E064E277E00E9421482DB73EB706
:10357000285030400FB6F8943EBF0FBE2DBFEDB7B8
:10358000FEB7319685E597E0ADB7BEB712969C932E
:103590008E93119789EE92E09383828380E790E087
:1035A0009583848382EB91E0978386830E94E9353B
:1035B00081E0EDB7FEB7389670C02DB73EB7285002
:1035C00030400FB6F8943EBF0FBE2DBFEDB7FEB72B
:1035D000319685E597E0ADB7BEB712969C938E9372
:1035E00011978FE692E09383828380E790E0958342
:1035F000848382EB91E0978386830E94E935EDB75F
:10360000FEB738960FB6F894FEBF0FBEEDBF80919F
:103610002E02851531F4442061F48091350288230F
:1036200041F010925D0710925E0710925F071092B2
:10363000600781E0E5960FB6F894DEBF0FBECDBF00
:10364000CF91DF911F910F91FF90EF90DF90CF907E
:10365000BF90AF909F908F907F906F905F904F90B2
:10366000089500D000D000D0EDB7FEB7319685E5C3
:1036700097E0ADB7BEB712969C938E9311978BE9E6
:1036800092E09383828380E790E0958384830E9415
:10369000E93581E0EDB7FEB736960FB6F894FEBF78
:1036A0000FBEEDBFC7CF0F931F93DF93CF93CDB75F
:1036B000DEB7C058D0400FB6F894DEBF0FBECDBF06
:1036C0008C010D5F1F4FC8010E94A919882309F4BE
:1036D00040C0C8018E010F5F1F4FB80140E820E4D1
:1036E00031E00E944750882341F0C8010E94935066
:1036F00080E890E0B8010E9421482DB73EB72850DD
:1037000030400FB6F8943EBF0FBE2DBFEDB7FEB7E9
:10371000319685E597E0ADB7BEB712969C938E9330
:1037200011978AE593E09383828380E790E0958305
:10373000848382EB91E0978386830E94E93581E060
:103740002DB73EB7285F3F4F0FB6F8943EBF0FBE70
:103750002DBFC058DF4F0FB6F894DEBF0FBECDBFF0
:10376000CF91DF911F910F9108958F929F92AF9209
:10377000BF92CF92DF92FF920F931F93DF93CF936D
:1037800000D000D0CDB7DEB773E0C72ED12CC80E65
:10379000D91EC6010E94A919882309F4B3C083E782
:1037A00089831A821B821C8210E062E0862E912C93
:1037B0008C0E9D1E5E010894A11CB11C1AC0812FA5
:1037C00090E0B4014AE050E00E94E509C60164E2DD
:1037D00077E040E395010E944750882349F084E256
:1037E00097E00E949350812F64E277E00E94554752
:1037F0001F5F8091520C181710F38DE68983FF2408
:1038000052E0852E912C8C0E9D1E5E010894A11C09
:10381000B11C1AC00F2D10E0C801B4014AE050E0FD
:103820000E94E509C60164E277E040E395010E9449
:103830004750882341F084E297E00E94E108075A4C
:10384000134FD8018C93F3948091510CF81610F318
:103850000E94964789E68983FF2442E0842E912CBA
:103860008C0E9D1E5E010894A11CB11C1AC00F2D68
:1038700010E0C801B4014AE050E00E94E509C60129
:1038800064E277E040E395010E944750882341F0CD
:1038900084E297E00E94E108015A134FF801808307
:1038A000F3948091510CF81610F30E947F472DB7C6
:1038B0003EB7285030400FB6F8943EBF0FBE2DBF24
:1038C000EDB7FEB7319685E597E0ADB7BEB7129676
:1038D0009C938E9311978DEA9BE09383828380E77C
:1038E00090E09583848382EB91E0978386830E94A6
:1038F000E93581E0EDB7FEB738960FB6F894FEBF14
:103900000FBEEDBF0F900F900F900F90CF91DF91F2
:103910001F910F91FF90DF90CF90BF90AF909F903D
:103920008F9008958F929F92AF92BF92CF92DF9225
:10393000EF92FF920F931F93CF93DF93EC017A01E5
:103940008B01CB01BA010E94EA434C01C801B701C7
:103950000E94E4435C018889882309F481C0D880EF
:10396000D7FE21C0C98021E02C15E8F4C801B701B9
:1039700020E831E541E050E00E94995CCA01B901BC
:103980002C2D30E040E050E00E94995C2FE7D222DD
:103990002D2D30E040E050E0621773078407950753
:1039A00009F05EC031C0C801B7010E94D843288128
:1039B00030E090E0059667E070E00E94865C02C00F
:1039C000359527958A95E2F720FF4AC0C801B701CF
:1039D0000E94DE43D82E888187FF16C08981882304
:1039E00019F4D0FE11C03CC0813071F48FE1D816BB
:1039F000B9F12DE1D21609F042C0C801B7010E9409
:103A0000D2430297E1F52CC08CE390E0889E9001B0
:103A1000899E300D989E300D11242A0D3B1D4A8140
:103A20005B8124173507E0F08C819D818217930715
:103A3000B8F0EE81FF81309799F0241B350B40E000
:103A4000C901BF010E94725C6E9FC0016F9F900D03
:103A50007E9F900D11248217930719F441E001C055
:103A600040E0842FDF91CF911F910F91FF90EF9055
:103A7000DF90CF90BF90AF909F908F900895D0FC33
:103A8000C3CFEECF982F9B0180916107981768F400
:103A900061E1969FB001112462597B4FC90141E158
:103AA00050E028E53AE00E9461090895CF92DF9244
:103AB000EF92FF920F931F93DF93CF93CDB7DEB7B3
:103AC00062970FB6F894DEBF0FBECDBF8C010D5FBD
:103AD0001F4FC8010E949350C80164E277E040E3A1
:103AE00024E431E00E944750882309F42BC184E28A
:103AF00097E00E94E1087C012FEF8F3F92070CF4C2
:103B000021C18091610790E0E816F9060CF01AC116
:103B10008DB79EB708970FB6F8949EBF0FBE8DBFA6
:103B2000EDB7FEB7319605E517E0ADB7BEB7129613
:103B30001C930E93119780E099E09383828380E732
:103B400090E09583848387E391E0978386830E9446
:103B5000E935EDB7FEB738960FB6F894FEBF0FBE45
:103B6000EDBF0E940713109258071092570786ED79
:103B700093E090935A078093590790935C07809342
:103B80005B072DB73EB72A5030400FB6F8943EBFC2
:103B90000FBE2DBFEDB7FEB73196ADB7BEB71296CB
:103BA0001C930E93119781EE98E09383828380910A
:103BB000510C84831582F782E6828091D602808739
:103BC00011860E94E935EDB7FEB73A960FB6F89424
:103BD000FEBF0FBEEDBFFFEFEF16FFEFFF0609F4CC
:103BE0008FC08E2D7E010894E11CF11CB7010E944C
:103BF000421D8A81823018F0C7010E946A112DB7D8
:103C00003EB7225130400FB6F8943EBF0FBE2DBFD5
:103C1000EDB7FEB7319605E517E0ADB7BEB7129622
:103C20001C930E93119782EC98E093838283898989
:103C3000848315828981868317828A818087118691
:103C40008B819C81938782878D819E8195878487D4
:103C50008F8198859787868789859A85918B808BB8
:103C60000E94E93590E0EDB7FEB772960FB6F89472
:103C7000FEBF0FBEEDBF6801EEEBEE2EE8E0FE2EBC
:103C80008E01055F1F4F22C000D000D000D0EDB7DD
:103C9000FEB73196ADB7BEB71196CC92119712967A
:103CA000DC92F382E282D801A90FB11D8C9184834A
:103CB00015829A8B0E94E9359A899F5FEDB7FEB70E
:103CC00036960FB6F894FEBF0FBEEDBF8091510C33
:103CD0009817D0F200D000D085E597E0ADB7BEB719
:103CE00012969C938E9311978BEB98E014969C936D
:103CF0008E9313970E94E9350F900F900F900F90BD
:103D000000D000D000D0EDB7FEB7319685E597E042
:103D1000ADB7BEB712969C938E9311978AE898E040
:103D20009383828380E890E0958384830E94E935C1
:103D300081E0EDB7FEB736960FB6F894FEBF0FBE22
:103D4000EDBF01C080E062960FB6F894DEBF0FBEF3
:103D5000CDBFCF91DF911F910F91FF90EF90DF903A
:103D6000CF9008952F923F924F925F926F927F92E1
:103D70008F929F92AF92BF92DF92EF92FF920F933A
:103D80001F93DF93CF93CDB7DEB761970FB6F8944B
:103D9000DEBF0FBECDBF00D000D000D0EDB7FEB764
:103DA000319605E517E0ADB7BEB712961C930E939A
:103DB000119784E09AE0938382838FEC90E095835F
:103DC00084830E94E93500D000D0EDB7FEB731966C
:103DD000ADB7BEB712961C930E9311978AED99E07A
:103DE0009383828380916107848315828091510C33
:103DF0008683178285E390E0918780870E94E9356A
:103E0000FF24EDB7FEB73A960FB6F894FEBF0FBE8B
:103E1000EDBF4E010894811C911CD02EE12E1BE0B9
:103E2000212E312C2C0E3D1EBBEB4B2EB9E05B2E10
:103E3000ADEB6A2EA9E07A2EF6EDAF2EF3E0BF2EA1
:103E4000ACC08F2DB4010E94421D8A81823018F0CF
:103E5000C4010E946A118DB79EB742970FB6F894BD
:103E60009EBF0FBE8DBFEDB7FEB73196ADB7BEB7E3
:103E70001196DC9211971296EC9284EC99E0938360
:103E800082838989848315828981868317828A81C6
:103E9000808711868B819C81938782878D819E810B
:103EA000958784878F8198859787868789859A8566
:103EB000918B808B0E94E93510E0ADB7BEB752966A
:103EC0001DC000D000D000D0EDB7FEB73196ADB721
:103ED000BEB71196DC9211971296EC9280EC99E0A5
:103EE00093838283D101A10FB11D8C9184831582AC
:103EF0000E94E9351F5FADB7BEB716960FB6F894AE
:103F0000BEBF0FBEADBF8091510C1817D0F20F2D60
:103F100010E08091610790E001970817190749F0B8
:103F200000D000D0EDB7FEB7D182E2827482638206
:103F30000EC000D000D0ADB7BEB71196DC9211977D
:103F40001296EC92129714965C924E9213970E94DE
:103F5000E9350F900F900F900F90037010700330A1
:103F60001105D1F480915B0790915C07209159076E
:103F700030915A07821B930B60E140E00E94C630EB
:103F80001092580710925707B0925A07A0925907FB
:103F9000B0925C07A0925B07F39480916107F816DA
:103FA00008F44FCF00D000D085E597E0EDB7FEB71D
:103FB0009283818388EB99E0948383830E94E9351F
:103FC0000F900F900F900F9081E061960FB6F894CC
:103FD000DEBF0FBECDBFCF91DF911F910F91FF903C
:103FE000EF90DF90BF90AF909F908F907F906F90F9
:103FF0005F904F903F902F9008952F923F924F9255
:104000005F926F927F928F929F92AF92BF92CF9268
:10401000DF92EF92FF920F931F93DF93CF93CDB771
:10402000DEB761970FB6F894DEBF0FBECDBF8DB778
:104030009EB70C970FB6F8949EBF0FBE8DBFEDB71D
:10404000FEB7319605E517E0ADB7BEB712961C93E3
:104050000E9311978EE79BE0938382838091610793
:10406000848315828091510C868317828091D602B9
:104070008087118685E390E0938782870E94E935E7
:10408000DD24EDB7FEB73C960FB6F894FEBF0FBE29
:10409000EDBF4E010894811C911CC02E012F2BE016
:1040A000222E312C2C0E3D1E4C2C512E9AE5692EC1
:1040B0009BE0792E86EDA82E83E0B82E9AC08D2D38
:1040C000B4010E94421D8A81823018F0C4010E940E
:1040D0006A11ED2CFF248DB79EB744970FB6F89464
:1040E0009EBF0FBE8DBFEDB7FEB73196ADB7BEB761
:1040F0001196CC92119712960C9381E69BE09383D4
:104100008283F582E4828989868317828981808708
:1041100011868A81828713868B819C81958784870B
:104120008D819E81978786878F819885918B808BE3
:1041300089859A85938B828B0E94E93510E0ADB713
:10414000BEB754961DC000D000D000D0EDB7FEB76A
:104150003196ADB7BEB71196CC92119712960C93CB
:104160008DE59BE093838283D101A10FB11D8C91DA
:10417000848315820E94E9351F5FADB7BEB71696DE
:104180000FB6F894BEBF0FBEADBF8091510C18178B
:10419000D0F200D000D0EDB7FEB7418252827482D7
:1041A00063820E94E935F3E0EF22FF240F900F9025
:1041B0000F900F9083E0E816F104D1F480915B0733
:1041C00090915C072091590730915A07821B930BFD
:1041D00060E140E00E94C6301092580710925707E5
:1041E000B0925A07A0925907B0925C07A0925B0761
:1041F000D39480916107D81608F461CF00D000D025
:1042000085E597E0ADB7BEB712969C938E93119754
:104210008FE49BE014969C938E9313970E94E9354C
:104220000F900F900F900F9061960FB6F894DEBF2D
:104230000FBECDBFCF91DF911F910F91FF90EF90F7
:10424000DF90CF90BF90AF909F908F907F906F90B6
:104250005F904F903F902F9008952F923F924F92F2
:104260005F926F927F928F929F92AF92BF92CF9206
:10427000DF92EF92FF920F931F93DF93CF9300D0C3
:10428000CDB7DEB78C010D5F1F4FC8010E94935060
:104290000E94FD445B016C010E94C9432C01C601D0
:1042A000B5010E94D2433C01C601B5010E94DE4324
:1042B0004C01C601B5010E94EA439A838983C60175
:1042C000B5010E94E4431C01C80164E277E040E3C9
:1042D00028E431E00E944750882361F084E297E0AF
:1042E0000E94E1084C01009729F4C601B5010E9423
:1042F000DE434C01C80164E277E040E32AE431E0A8
:104300000E944750882329F084E297E00E94E10848
:104310003C01C80164E277E040E32CE431E00E9414
:104320004750882329F084E297E00E94E1082C019D
:1043300000D000D000D0EDB7FEB7319655E5E52EA0
:1043400057E0F52EADB7BEB71296FC92EE921197DC
:1043500084E598E09383828380E790E0958384836B
:104360000E94E935EDB7FEB736960FB6F894FEBF5A
:104370000FBEEDBF0E940713109258071092570707
:1043800086ED93E090935A078093590790935C07CA
:1043900080935B072DB73EB72A5130400FB6F89493
:1043A0003EBF0FBE2DBF0DB71EB70F5F1F4FADB77E
:1043B000BEB71296FC92EE9211978DEF97E0F8013E
:1043C0009383828380919702848315828091A502D2
:1043D000868317828091C8028087118680919E0211
:1043E000828713868091AC02848715868091B30200
:1043F00086871786C601B50120E831E541E050E027
:104400000E94995CD80151963C932E9350978CE36F
:1044100090E0E981FA819C01E29FC001E39F900D49
:10442000F29F900D1124820D931D53969C938E93B1
:10443000529755969C928E92549757967C926E9274
:10444000569759965C924E9258970E94E9354DB70F
:104450005EB74A5E5F4F0FB6F8945EBF0FBE4DBFAA
:10446000ADB7BEB71296FC92EE92119781EF97E02E
:1044700014969C938E9313970E94E93500E00F9059
:104480000F900F900F90BE2CEF2C4DEEC42E47E0F6
:10449000D42E21C000D000D000D0EDB7FEB73196A9
:1044A000ADB7BEB71196BC9211971296EC92D3821B
:1044B000C282A02FB0E0A75AB34F8C91848315829B
:1044C0000E94E9350F5FEDB7FEB736960FB6F89448
:1044D000FEBF0FBEEDBF8091510C35E5832E37E056
:1044E000932E0817B8F200D000D0ADB7BEB7129621
:1044F0009C928E92119789EE97E014969C938E93DE
:1045000013970E94E9350F900F900F900F900E9423
:10451000FD1F00D000D000D0EDB7FEB73196ADB78B
:10452000BEB712969C928E92119781EC97E093837E
:10453000828380E890E0958384830E94E935EDB71B
:10454000FEB736960FB6F894FEBF0FBEEDBF81E002
:104550000F900F90CF91DF911F910F91FF90EF90EF
:10456000DF90CF90BF90AF909F908F907F906F9093
:104570005F904F903F902F9008950F931F938DB7AA
:104580009EB708970FB6F8949EBF0FBE8DBFEDB7CC
:10459000FEB7319605E517E0ADB7BEB712961C938E
:1045A0000E93119785E399E09383828380E790E0EF
:1045B0009583848387E391E0978386830E94E9351E
:1045C0008DB79EB708960FB6F8949EBF0FBE8DBFED
:1045D0000E940713109258071092570786ED93E038
:1045E00090935A078093590790935C0780935B07D9
:1045F0000E94FD1F00D000D000D0EDB7FEB731966D
:10460000ADB7BEB712961C930E9311978DE099E04B
:104610009383828380E890E0958384830E94E935C8
:104620008DB79EB706960FB6F8949EBF0FBE8DBF8E
:1046300081E01F910F910895DF92EF92FF920F9307
:104640001F93DF93CF93CDB7DEB761970FB6F89482
:10465000DEBF0FBECDBF20916107821708F043C0B7
:10466000222309F440C090E001968C0174E0000F11
:10467000111F7A95E1F7080F191F02591B4F61E1CD
:10468000D62E7E010894E11CF11C13C0C701B801AD
:1046900041E150E028E53AE00E946109C8014197F4
:1046A000B70141E150E020E63AE00E94A3090F5E25
:1046B0001F4F209161072D9DC001112482599B4FEE
:1046C0000817190718F3215020936107F999FECFB5
:1046D0001FBA8CE694E092BD81BD20BD0FB6F89460
:1046E000FA9AF99A0FBE61960FB6F894DEBF0FBE24
:1046F000CDBFCF91DF911F910F91FF90EF90DF9091
:104700000895CF93DF93EC012396CE010E9493503E
:10471000CE010E94A919882309F450C0CE0164E299
:1047200077E040E324E431E00E944750882309F415
:1047300045C084E297E00E94E1089C018FEF2F3F83
:10474000380781F410926107F999FECF1FBA8CE601
:1047500094E092BD81BD10BC0FB6F894FA9AF99A14
:104760000FBE09C08091610790E02817390734F522
:10477000822F0E941C2300D000D000D0EDB7FEB7DE
:10478000319685E597E0ADB7BEB712969C938E93B0
:1047900011978FE598E09383828380E790E095837B
:1047A00084830E94E93581E02DB73EB72A5F3F4FF1
:1047B0000FB6F8943EBF0FBE2DBF01C080E0DF9161
:1047C000CF910895982F80916107981760F481E147
:1047D000989FC001112482599B4F41E150E020E68F
:1047E0003AE00E94A3090895BC01909161079533B6
:1047F000F0F481E1989FC001112482599B4F41E15F
:1048000050E020E63AE00E94A309209161072F5F63
:1048100020936107F999FECF1FBA8CE694E092BD10
:1048200081BD20BD0FB6F894FA9AF99A0FBE08958B
:10483000BF92CF92DF92EF92FF920F931F93DF937D
:10484000CF93CDB7DEB763970FB6F894DEBF0FBE38
:10485000CDBF7C018C010D5F1F4FC8010E9493509A
:10486000C8010E94A919882309F403C1C80164E2A0
:1048700077E040E324E431E00E944750882309F4C4
:10488000F8C084E297E00E94E1086C012FEF8F3FAF
:1048900092070CF4EEC08091610790E0C816D9062B
:1048A0000CF0E7C01A83098387E690E0E80EF91E52
:1048B0000DC0C8016EE471E043E050E00E9453096E
:1048C000009779F00F5F1F4F1A83098309811A81BE
:1048D000D8018C91882309F4CCC00E151F0548F32C
:1048E000C8C00D5F1F4F1A8309838E010F5F1F4FD2
:1048F000C8010E949F0E8B8BC8010E949F0E8B8364
:10490000C8010E949F0E8C83C8010E949F0E9E8347
:104910008D83C8010E949F0E98878F83C8010E94D3
:104920009F0E9A878987C8010E949F0E9C878B875C
:10493000FF24B02EE12E8E01035F1F4F09C08B2D87
:104940009E2D0E949F0EF801EF0DF11D8083F394C0
:104950008091510CF81698F306C0FC01EF0DF11D83
:104960001082F39402C0CE010D96B5E0BF15A8F7F2
:104970008C81823020F0CE0103960E943B1100D042
:1049800000D000D0EDB7FEB7319605E517E0ADB722
:10499000BEB712961C930E93119786EB97E0938304
:1049A000828380E790E0958384830E94E935EDB7A8
:1049B000FEB736960FB6F894FEBF0FBEEDBFBE0130
:1049C0006D5F7F4FFFEFCF16FFEFDF06C1F4CB0126
:1049D0000E94F42300D000D0ADB7BEB712961C934E
:1049E0000E93119789E997E014969C938E931397F1
:1049F0000E94E9350F900F900F900F9022C08C2DE0
:104A00000E94E22300D000D000D0EDB7FEB731966F
:104A1000ADB7BEB712961C930E9311978BE797E034
:104A2000938382830894C11CD11CD582C4820E94C6
:104A3000E935EDB7FEB736960FB6F894FEBF0FBE58
:104A4000EDBF00D000D085E597E0ADB7BEB71296B8
:104A50009C938E9311978AE597E014969C938E937E
:104A600013970E94E93581E00F900F900F900F90FF
:104A700001C080E063960FB6F894DEBF0FBECDBFD5
:104A8000CF91DF911F910F91FF90EF90DF90CF902A
:104A9000BF9008950E94D1470E94524CAAEEB8E000
:104AA00080E090E0FC01E659F84F108211821282FA
:104AB0001382FC01E65DF74F10821182128213828D
:104AC0001D920496803C910569F70895EF92FF923C
:104AD0000F931F93CF93DF93EC012396CE010E9497
:104AE000A919882309F407C1CE0164E277E040E305
:104AF00022E531E00E944750882311F00E944A25A8
:104B0000CE0164E277E040E326E531E00E944750C1
:104B1000882309F44CC084E297E00E94E10818164B
:104B200019060CF044C02DB73EB7285030400FB6E0
:104B3000F8943EBF0FBE2DBFEDB7FEB7319605E529
:104B400017E0ADB7BEB712961C930E9311978CE980
:104B500093E09383828380E790E09583848384E16C
:104B600090E0978386830E94E9350F900F900F9015
:104B70000F90EDB7FEB7128301838FE893E0948323
:104B800083830E94E9350F900F900F900F908091D2
:104B90005B0790915C072091590730915A07821B5F
:104BA000930B61E140E00E94C6300E942A47CE018B
:104BB00064E277E040E32AE531E00E944750882331
:104BC00099F080912407813339F480914F0C80FD56
:104BD0000BC00E94B94C08C0803331F480914F0C57
:104BE00080FF02C00E94AF4CCE0164E277E040E358
:104BF0002DE531E00E9447508823E9F08091240799
:104C0000813351F480914F0C84FD15C00E944A25D8
:104C100080914F0C80610BC0803369F480914F0C00
:104C200084FF09C00E944A2580914F0C8F7E80939B
:104C30004F0C0E94F34BCE0164E277E040E320E6A4
:104C400031E00E944750882351F184E297E00E94AE
:104C5000E108EC0118161906F4F40E94FD447B01EA
:104C60008C01BE01882777FD8095982F20E13EE0DA
:104C700040E050E00E94475CE60EF71E081F191F37
:104C8000E092650CF092660C0093670C1093680C30
:104C90000E94A54C04C0009771F50E94934C2DB75B
:104CA0003EB7285030400FB6F8943EBF0FBE2DBF20
:104CB000EDB7FEB7319685E597E0ADB7BEB7129672
:104CC0009C938E93119782E893E09383828380E78D
:104CD00090E09583848382EB91E0978386830E94A2
:104CE000E93581E0EDB7FEB738960FB6F894FEBF10
:104CF0000FBEEDBF01C080E0DF91CF911F910F91FA
:104D0000FF90EF900895BF92CF92DF92EF92FF92C3
:104D10000F931F93DF93CF9300D0CDB7DEB77C0105
:104D20008C010D5F1F4FC8010E949350C8010E9463
:104D3000A919882309F4A0C01A83098327E630E063
:104D4000E20EF31E0DC0C80163E671E043E050E0DF
:104D50000E945309009779F00F5F1F4F1A83098350
:104D600009811A81D8018C91882309F485C00E1518
:104D70001F0548F381C00D5F1F4F1A8309830E94EE
:104D80004A25FF2400E014E0EE246E010894C11CC3
:104D9000D11CBEEFBB2E37C0C6010E949F0EF999F1
:104DA000FECF1FBA12BD01BD90BD0FB6F894FA9A9E
:104DB000F99A0FBEF999FECF1FBA0F5F1F4F12BDB0
:104DC00001BD0150104080BD0FB6F894FA9AF99ACF
:104DD0000FBE0097A9F02F2D30E0F901EE0FFF1F55
:104DE000EE0FFF1FE65DF74FA0E0B0E080839183F8
:104DF000A283B3832651374FF901B082EE24E394A6
:104E0000F3940E5F1F4F8091520CF81608F4C4CF34
:104E1000EE2031F00E94FD44409197020E94760AF4
:104E20002DB73EB7285030400FB6F8943EBF0FBEA6
:104E30002DBFEDB7FEB7319685E597E0ADB7BEB7AC
:104E400012969C938E93119782E499E093838283C8
:104E500080E790E09583848382EB91E0978386835B
:104E60000E94E93581E0EDB7FEB738960FB6F894A9
:104E7000FEBF0FBEEDBF01C080E00F900F90CF913D
:104E8000DF911F910F91FF90EF90DF90CF90BF9037
:104E900008952F923F924F925F926F927F928F92DE
:104EA0009F92AF92BF92CF92DF92EF92FF920F93B9
:104EB0001F93DF93CF9300D000D0CDB7DEB7109112
:104EC000A50290914F0C292F21702A83892E82945C
:104ED0003FE0832231E0832291FD0CC08091BA0231
:104EE000882311F4EE2408C0E92EE694E69441E00C
:104EF000E42211F0EE24E3940E94FD445B016C0176
:104F00009924212E3324A5C0892D90E0FC01E15A7B
:104F1000F34F3081FC01ED5AF34F2081A92DAA0FE8
:104F2000AA0FAA0FA98300E010E0422E5524632E99
:104F30007724882009F086C0F980F00EEF2DF0E08C
:104F4000FC83EB83E651F74FE081EE3F09F47AC032
:104F5000FA81FF2361F0EE2009F474C0C301002E32
:104F600002C0959587950A94E2F780FD6BC0C20157
:104F7000002E02C0959587950A94E2F780FF47C0FE
:104F80008F2D60E00E94AD478B819C810196281691
:104F9000390611F1F0926207EB81FC81E651F74F7F
:104FA000808180936307EB81FC81EE0FFF1FEE0F82
:104FB000FF1FE659F84F808191819501281B390B1D
:104FC0003093650720936407A0926607B092670745
:104FD000C0926807D0926907EB81FC81EE0FFF1F3A
:104FE000EE0FFF1FDF01A659B84F1D921D921D92B3
:104FF0001C921397E65DF74F108211821282138282
:105000008B819C818651974FDC011C921BC0EE2343
:10501000C9F0EB81FC81EE0FFF1FEE0FFF1FDF01D8
:10502000A659B84F1D921D921D921C921397E65DD2
:10503000F74F1082118212821382EB81FC81E651BC
:10504000F74F10820F5F1F4F0830110509F071CF25
:1050500093948091510C981608F456CF0F900F90AE
:105060000F900F90CF91DF911F910F91FF90EF90D4
:10507000DF90CF90BF90AF909F908F907F906F9078
:105080005F904F903F902F900895EF92FF920F9373
:105090001F939B01AC0180911A0990911B09A0916B
:1050A0001C09B0911D090097A105B10549F4209391
:1050B0001A0930931B0940931C0950931D0954C0D1
:1050C00079018A01E81AF90A0A0B1B0BD801C701FA
:1050D000CD97A105B10508F447C020931A09309374
:1050E0001B0940931C0950931D0983E799E00E9416
:1050F000A7320E94C9567B018C010E94E02D0E94BC
:10510000F43283E799E00E946835882361F40E94B5
:10511000C9566E197F09800B910B683C710581059A
:10512000910558F319C08091500C8F708093500CEA
:105130008091500C82958F7090E00397ACF0809135
:105140008902882389F060919E0370919F0385EA0C
:1051500091E00E94EE4F08C08091500C982F907FF4
:10516000905F8F70892BE2CF1F910F91FF90EF908E
:105170000895EF92FF920F931F939B01AC018091D2
:105180003502882309F443C08091500C82958F70BA
:1051900009F03DC080914F0C83FD39C080915D07BF
:1051A00090915E07A0915F07B09160070097A105FD
:1051B000B10569F079018A01E81AF90A0A0B1B0B9B
:1051C000D801C70181589145A140B04000F120931A
:1051D0005D0730935E0740935F07509360078EEB47
:1051E0009CE061E00E9442490E945F0E7B018C01BD
:1051F000611571058105910551F00E94D04480919F
:105200004F0C85FF04C0C801B7010E94D0461F9112
:105210000F91FF90EF9008950E94C84E0E94154D87
:105220000E941B0B9091820280E020917B02820FF2
:10523000911D90939F0380939E036CE370E080E048
:1052400090E00E94C74480914F0C85FD03C080E030
:1052500090E002C080EF96E40E94704564EF71E038
:1052600080E090E00E94D75680E00E947E4E8BED59
:105270009CE061E00E94424981EC99E060E00E947C
:10528000113F882329F480914F0C806480934F0C48
:105290008DEC9CE061E00E94424960919E03709118
:1052A0009F0385EA91E00E94EE4F882321F08091D0
:1052B000500C8F7004C08091500C8F70806180936F
:1052C000500C64EF71E080E090E00E94D7560E949D
:1052D000524C0E94FD446093690C70936A0C809359
:1052E0006B0C90936C0C08951F93CF93DF9382E027
:1052F0000E94B348182FC82FD0E086FF54C00E94E8
:10530000FD446093690C70936A0C80936B0C9093CE
:105310006C0C8091EB026FEF70E0681B71098CE000
:105320000E947258CE018F7090708230910589F082
:105330008430910501F10197B1F517FF03C00E9478
:10534000B94C31C060910402709105028BE699E07E
:1053500009C017FF03C00E94AF4C25C083E799E046
:1053600060E070E00E94AB4B60ED77E080E090E0A1
:105370000E94D75618C017FF06C081E00E94B348AC
:105380000E942A4710C02091500C822F8F7090E00D
:105390006091510C019670E00E94865C8F70207FB6
:1053A000282B2093500CDF91CF911F9108952F92BD
:1053B0003F924F925F926F927F928F929F92AF92A5
:1053C000BF92CF92DF92EF92FF920F931F93DF93E2
:1053D000CF93CDB7DEB7AA970FB6F894DEBF0FBE56
:1053E000CDBF209197022C8B3091A5023B8B0E9460
:1053F000E02D0E94F43290931F0980931E090097BC
:1054000021F080569C4F0E947E150E9474290E94B4
:10541000FD445B016C018091240990912509A091C4
:105420002609B09127098A159B05AC05BD0509F42D
:10543000D9C2A0922409B0922509C0922609D0921F
:10544000270980E00E947E4E80914F0C2091650CD0
:105450003091660C4091670C5091680C81FF08C038
:10546000A216B306C406D50650F00E94934C07C09E
:10547000A216B306C406D50610F40E94A54C80916E
:10548000690C90916A0CA0916B0CB0916C0C009718
:10549000A105B105C9F04E96A11DB11D8A159B0548
:1054A000AC05BD0588F48091F2026FEF70E0681BD7
:1054B00071098CE00E9472581092690C10926A0C6B
:1054C00010926B0C10926C0C0E94FC4880914F0C57
:1054D00084FDC4C083FF04C04C89442309F0BEC0CE
:1054E000C601B5012CE330E040E050E00E94995C39
:1054F00079018A018091200990912109A0912209C6
:10550000B0912309E816F9060A071B0709F4A6C09B
:10551000E0922009F09221090093220910932309B7
:10552000662410E09B89892F90E09AA789A78AC0FA
:10553000862DBE016F5F7F4F0E94421DCE010196F6
:10554000B601A5010E94921C882309F47AC029851E
:105550003A852115310509F474C0A091510CAE8B28
:1055600077241A8A190144245524B62DBF5FB8A7A1
:1055700053C08A89880DE82EFF24C7010196E9A54A
:10558000FAA5E817F907E1F1ACA1BDA18C9190E073
:10559000082C02C0959587950A94E2F780FD30C0EB
:1055A000EEA1FFA1808190E0082C02C0959587951F
:1055B0000A94E2F780FF24C08701000F111F000F3B
:1055C000111F065D174F6091C80270E080E090E007
:1055D000A20191010E94475C24E630E040E050E0E7
:1055E0000E94995CD8012D933D934D935C93139742
:1055F000EAEEF8E0EE0EFF1EE8A5D701EC9311E00D
:105600000894811C911CF8E08F16910409F0B1CF29
:1056100073942A89285F2A8B3E89731690F4872D0C
:1056200090E088249924AC014D5A534F5DA34CA3BC
:10563000ABE0B0E0AC0FBD1FA80FB91FBFA3AEA376
:1056400098CF639480916107681608F471CF112395
:1056500029F0C601B5014C890E94760A80914F0C51
:1056600083FF52C14424FB89EF2FF0E0FC8FEB8FC6
:105670002B8921502D8F30E0C901880F991F880F89
:10568000991FAC014659584F5F8F4E8FDC01A65DC4
:10569000B74FB9A3A8A3F901E651F74FFBA3EAA3BB
:1056A00014C1842D90E0FC01ED5AF34F2081F42DBC
:1056B000FF0FFF0FFF0FFD8B66247724422F50E072
:1056C000588F4F8BDC01A75AB34FBA8FA98F5D88D3
:1056D000560C852C99241AEEE12E18E0F12EE80CD8
:1056E000F91CF7018081882309F44DC08401000F63
:1056F000111F000F111FF801E65DF74F80819181A6
:10570000A281B381A816B906CA06DB06E0F1852D91
:1057100060E00E94AD47C40101962B8D3C8D281797
:105720003907D1F050926207D7018C9180936307BB
:105730000659184FF801808191819501281B390B7A
:105740003093650720936407A0926607B0926707BD
:10575000C0926807D0926907F401EE0FFF1FEE0FA9
:10576000FF1FDF01A659B84F1D921D921D921C927A
:105770001397E65DF74F1082118212821382F401B3
:10578000E651F74F10828F89988D062C02C09595AF
:1057900087950A94E2F780FD8FC09401220F331F92
:1057A000220F331F89010659184FF801808191811A
:1057B000A281B381A816B906CA06DB0608F47CC02C
:1057C0006AE2262E68E0362E220E331EF101808119
:1057D0009181A281B381A816B906CA06DB0608F03A
:1057E0006BC0852D61E00E94AD47FB89FF2309F462
:1057F00063C0C40101962B8D3C8D2817390709F42D
:105800005BC0A98DBA8D8C9190E0062C02C0959555
:1058100087950A94E2F780FF4FC0BC89BB2309F447
:105820004BC080914F0C84FD47C08091AC02F801C1
:105830002081318142815381280F311D411D511D2D
:10584000AE8DBF8D2D933D934D935C9313978091B7
:10585000B302E82EFF2400E010E084EC9FEFAFEFEE
:10586000BFEFE80EF91E0A1F1B1FF1018081918115
:10587000A281B381E80EF91E0A1F1B1FA8A1B9A1BE
:10588000ED92FD920D931C931397EAEEF8E08E0EC5
:105890009F1ED4018C91EAA1FBA18083A216B306BE
:1058A000C406D50648F0AE14BF04C006D10620F4E5
:1058B0008D8D61E00E94AD470894611C711CF8E079
:1058C0006F16710409F003CF43948091510C481670
:1058D00008F4E7CE0E9449270E94524C3091520CA6
:1058E000EAE2F8E020E00DC081919191A191B1919F
:1058F0000197A109B1098E5F9F4FAF4FBF4F20F0B5
:105900002F5F231788F363C05B89552369F080916B
:105910004F0C84FF09C01091520C40E021E030E0B0
:105920008B89682F70E02EC09C899923A1F331C028
:10593000842F90E06217730711F1DC0153E0B695F4
:10594000A7955A95E1F7542F5770FD01ED5AF34F83
:10595000808190E0052E02C0959587950A94E2F724
:1059600080FF0DC0A75AB34F8C9190E002C095956F
:1059700087955A95E2F780FF02C061E006C04F5F4D
:105980002F5F3F4F4117A0F260E08B8981500E944A
:10599000AD470E9449270E94524CC601B50123E041
:1059A00030E040E050E00E94995C9B01AC01255C36
:1059B0003C4F81E0D9016C910E94174BC601B501A3
:1059C0000E944528C601B5010E94B9280BC00E945B
:1059D000D14780914F0C877F80934F0CB091A502E7
:1059E000BB8B92CFAA960FB6F894DEBF0FBECDBF89
:1059F000CF91DF911F910F91FF90EF90DF90CF90AB
:105A0000BF90AF909F908F907F906F905F904F90DE
:105A10003F902F90089580912A0961E00E94CB5712
:105A200078940895FF920F931F93082F162FF42E4A
:105A3000F89480912A0960E00E94CB571F71102BC7
:105A40001EBD0DB407FEFDCFFEBC0DB407FEFDCF9D
:105A50000E940B2D1F910F91FF9008951F93182FF7
:105A6000282F30E02076307080912B0990E02817A5
:105A7000390799F080EA6FE143E00E94122D412F2F
:105A8000407640932B0950E085E0559547958A95DF
:105A9000E1F780E86FE10E94122D1F9108950F93A6
:105AA0001F93182F062F0E942E2D80E4612F402F68
:105AB0000E94122D1F910F9108950F931F93182F7D
:105AC000072F0E944F2D812F8F5F602F0E944F2D37
:105AD0001F910F91089588E360EB0E944F2D089568
:105AE00088E361EB0E944F2D08950F931F93182FA9
:105AF000062FF89480912A0960E00E94CB57802FEE
:105B00008F71812B8EBD0DB407FEFDCF1EBC0DB471
:105B100007FEFDCF07FF04C01EBC0DB407FEFDCF7E
:105B20001EB50E940B2D812F1F910F9108951F9379
:105B3000182F0E942E2D80E0612F0E94752D1F913D
:105B4000089584ED61E10E944F2D82ED61E00E9495
:105B50004F2D8AEE0E94972D80FDFBCF82ED60E0F5
:105B60000E944F2D89ED0E94972D90E09695879584
:105B700096958795817008950F931F93CF93DF9328
:105B8000EC018B01F89480912A0960E00E94CB57C8
:105B90008AE38EBD0DB407FEFDCF09C01EBC0DB457
:105BA00007FEFDCF8EB5F80181938F0121972097D5
:105BB000A9F70E940B2DDF91CF911F910F910895AE
:105BC0000F931F93DF93CF9300D000D000D0CDB7B9
:105BD000DEB789E30E94972D882319F400E010E0D6
:105BE00048C060912C0970912D0980E00E945D2DC4
:105BF00086E090E0BE016F5F7F4F0E94BC2D8981DF
:105C00009A8190932D0980932C092B813C81E091FE
:105C10002809F09129098D8187FD03C000E010E07B
:105C20000EC0245030408F01015010402017310722
:105C300008F48901C80160EA73E00E94BC2DF801F4
:105C4000E056FC4F108260912C0970912D098CE078
:105C50006130780724F08CE06FEF7BE003C0615087
:105C600070408CE00E945D2D80E86EE140E40E946F
:105C7000122DC80126960FB6F894DEBF0FBECDBF19
:105C8000CF91DF911F910F9108950F931F93CF93A1
:105C9000DF938C01EB01F89480912A0960E00E9467
:105CA000CB578AE78EBD0DB407FEFDCF08C08881B3
:105CB0008EBD0DB407FEFDCF219601501040011599
:105CC0001105A9F70E940B2DDF91CF911F910F9124
:105CD0000895CF93DF93EC010FC08CE10E94972DC4
:105CE00081FF0AC080E86FE140E80E94122D80EA3F
:105CF0006FE140E80E94122D80E06FE10E94752D57
:105D000083FDEBCF82E060E07CE00E945D2DBE0170
:105D10006050744F86E00E945D2D8AE760E040E0AD
:105D20000E94122DCE0160EA73E00E94452E80E8A9
:105D30006FE148E00E94122DDF91CF91089584E039
:105D400061E00E948C5784E061E00E94CB5785E0BF
:105D500061E00E948C5787E061E00E948C5786E0EA
:105D600060E00E948C5785E061E00E94CB5785E09F
:105D700060E00E94CB5787E060E00E94CB5780E54F
:105D80008CBD8DB581608DBD08951F93CF93DF933A
:105D9000EB01142F90932909809328090CB406FC79
:105DA00002C00E949F2E10932A09812F61E00E9459
:105DB0008C570E940B2D8FEF60E04FEF0E94122D49
:105DC00062E070E080E090E00E94D75680E06DE1F4
:105DD0000E94752D8823D1F310922D0910922C0961
:105DE00088E060E070E00E945D2D8CE060E070E093
:105DF0000E945D2D8AE06FEF7BE00E945D2D84E0C4
:105E000060E07CE00E945D2D86E06FEF71E10E9412
:105E10005D2D0E94702D88E26FE370E30E945D2D7E
:105E200080E369EF77EF0E945D2D80EC6DE00E94CA
:105E30004F2D81EC60E00E944F2D80E862EC42E340
:105E40000E94122D86EC62E17CE00E945D2D84ECC4
:105E500062E10E944F2D8AEC6CED75E00E945D2D91
:105E600084EE68810E944F2D85EE69810E944F2D3E
:105E700082EE6A810E944F2D83EE6B810E944F2D2E
:105E800080EE6C810E944F2D81EE6D810E944F2D1E
:105E900084ED60E10E944F2D86ED60E071E00E948C
:105EA0005D2D8AEE0E94972D80FDFBCF8FE10E9431
:105EB0002E2D80E86BE140EC0E94122D80E86FE10E
:105EC00044E00E94122D82E70E94972D863008F050
:105ED0008F5FDF91CF911F910895DF92EF92FF9234
:105EE0000F931F93CF93DF93D82E862FBA012130C3
:105EF00041F4675F7F4F9B0140E050E06950704084
:105F00000EC0223029F020E030E040E050E007C031
:105F1000625070409B0140E050E06E5F7F4FE82E82
:105F2000FF2480EA93E0E80EF91E8B01E7010FC021
:105F3000F881E0E0898190E08E2B9F2BA0E0B0E01B
:105F4000280F391F4A1F5B1F229602501040023053
:105F5000110570F7CB018E7FD701A80FB91F681705
:105F6000790779F08C9190E0A0E0B0E0BA2FA92FEA
:105F7000982F882702C040E050E0280F391F4A1FA1
:105F80005B1FCA01AA27BB270097A105B10599F796
:105F9000C90180959095ED2DF0E0E056FC4F90837F
:105FA0008183DF91CF911F910F91FF90EF90DF9050
:105FB00008951092B8031092B90380E48093B4035B
:105FC0001092B5038093B60388E16EE044E150E09F
:105FD00020E00E946D2F0895282F662321F08091E4
:105FE000C5038617E1F48091C6038823C1F480912C
:105FF000C7038833A1F48091C3038B3781F4E22F68
:10600000F92F8091F20383838091F303828380913F
:10601000F40381838091F503808381E0089580E01B
:1060200008950F931F93BC0100EA13E0C8010E947A
:10603000D650C801069665E679E00E94D6501F91B9
:106040000F910895EF92FF920F931F937B010E948F
:1060500011300EEB13E0C801B7010E94DE50C801F9
:1060600004976BE679E00E94DE501F910F91FF903C
:10607000EF900895EF92FF920F931F93CF93DF93CA
:106080007C01EB018A0189E399E00E94223088813A
:10609000807F803E49F088819981AA81BB818F5F92
:1060A0009F4FAF4FBF4F31F480EA93E06EE373E050
:1060B0000E94D65088E08093AC031092AD038EEA24
:1060C00093E064EF7CE049E050E00E9426091092E2
:1060D000B00381E18093B7031093C4030093C50319
:1060E000F092C203E092C3031092C6031092C80359
:1060F0001092C903DF91CF911F910F91FF90EF9004
:106100000895EF92FF920F931F9306EA13E0C801E0
:106110000E94113074E1E72EF12CE00EF11EC8014F
:106120004896B7010E94DE50C7016BE679E00E94F5
:10613000DE500E94D92F1F910F91FF90EF9008958C
:10614000BC0181E080932E0983E799E00E94DE5034
:1061500008950F931F938C0188969093B0038093BA
:10616000B1030E94D92F1092D2031092D303045E80
:106170001F4F82E36AE1A80122E00E946D2FC8014F
:106180004A960E94692E1F910F910895FF920F93D6
:106190001F93CF93DF93EC01F62E042F10E0809134
:1061A000410990914209A0914309B09144092B2FD4
:1061B0003327442755272093C603A093C703909302
:1061C000C8038093C903F092CF03CE010E94A93087
:1061D0001F5F011720F79E0140E050E080914109C8
:1061E00090914209A0914309B0914409820F931FF5
:1061F000A41FB51F8093410990934209A0934309BE
:10620000B0934409DF91CF911F910F91FF900895B2
:10621000CF93DF939C01862F80618093CF036430FE
:1062200029F02115310511F421E030E09091C403EB
:106230008091C2038093C4039093C2039091C503DD
:106240008091C3038093C5039093C303C9ECD3E04B
:106250008881A901480F511D2C814C832883252F4B
:106260003327219753E0C53CD50791F71D861E863D
:1062700080E589871092B00388E28093B1030E9481
:10628000813084E08B871C8682E36AE14CE150E038
:1062900022E00E946D2F86E390E00E94692EDF913C
:1062A000CF91089580913F099091400960E00E944C
:1062B00008318091C60390E0A0E0B0E0BA2FA92F8A
:1062C000982F88272091C703820F911DA11DB11D12
:1062D000BA2FA92F982F88272091C803820F911DCC
:1062E000A11DB11DBA2FA92F982F88272091C9036E
:1062F000820F911DA11DB11D809341099093420908
:10630000A0934309B09344090895E82FA091B003E6
:10631000B091B103F091CE034091C40350E0292F16
:1063200030E04217530709F08EC08091C5038E17E5
:1063300009F089C08091CF03E82F81FF4EC01092F1
:10634000B0038CE28093B1030E94813082E180939C
:10635000CF039091C4038091C2038093C4039093B0
:10636000C2039091C5038091C3038093C5039093AA
:10637000C303E9ECF3E021E030E08081A901480F9C
:10638000511D44831082252F3327319753E0E53C7C
:10639000F50799F7158616861182128280910302FD
:1063A000838314828D5F8093030282E0818B84E07B
:1063B000828B95E0938B148A80E68187938788E7A8
:1063C000848782E36AE140E250E022E00E946D2F80
:1063D0008AE390E00E94692E36C084FF34C04F2FBC
:1063E00050E084E0559547958A95E1F79A2F80E033
:1063F0002B2F30E0282B392BCA01880F991F880FCB
:10640000991F281B390B2451304037FF02C020E070
:1064100030E03093400920933F09232B69F09A0123
:10642000220F331F220F331F2E5D3F4F68507040E5
:106430006217730740F009C0E0FF05C080E090E0FC
:1064400060E00E94083120E030E0C90108950F9318
:106450001F93DF93CF930F92CDB7DEB78C01045E0D
:106460001F4F1093B0030C511040802F845E809317
:10647000B10389830E94D92F085F1F4F1093C60371
:10648000898184518093C703085F1F4F88E26AE1C6
:10649000A80121E00E946D2FC8014A960E94692E32
:1064A0000F90CF91DF911F910F910895FF920F935D
:1064B0001F939C01F62E89E399E0B9010E942230D6
:1064C0000CEA13E088E08093AC031092AD03C8019E
:1064D000029664EF7CE049E050E00E9426098CE4DB
:1064E0008093B10381E18093B7030E94D92F10926A
:1064F000C4038BE78093C5038AE08093C203F092C4
:10650000C3031092C60388E38093C7031092C803A5
:106510001092C903025E1F4F80E3F80111928A9521
:10652000E9F7C8016BEA7DE04AE050E00E942609E5
:1065300088E26AE140E450E021E00E946D2F8AE5A4
:1065400090E00E94692E1F910F91FF900895EF92A5
:10655000FF920F931F93BC0189E399E00E942230C0
:106560000CEA13E038E0F32EF092AC031092AD0386
:10657000C801029664EF7CE049E050E00E942609E1
:1065800084E58093B103EE24E394E092B7030E9484
:10659000D92FF092C2031092C3031092C403109239
:1065A000C50385E08093C60380916E098093C7037D
:1065B0001092C803E092C903C8014E9662E470E0ED
:1065C00048E350E00E943C0984E262E240E450E08B
:1065D00020E00E946D2F82E690E00E94692E1F91BC
:1065E0000F91FF90EF900895DF92EF92FF920F933B
:1065F0001F93CF93DF93EC0180918309882319F0D7
:10660000CE010E94B237209709F0BFC080912E09B9
:106610008570F1F18091000290910102892BC1F502
:106620000E94A12D8823A1F18EE393E00E941130F6
:1066300088E08093AC03A6E0FA2EF092AD038EEAD8
:1066400093E06CEE7CE048E050E00E94260900EC0C
:1066500013E0D8011D92FA94E9F7C8010A9765E69C
:1066600079E00E94D650C801069663E779E00E945F
:10667000DE50C80104976BE679E00E94DE508091FD
:106680002E09886080932E098AE290E00E94692E8C
:1066900080910002909101020196909301028093F3
:1066A000000280912F09813009F002C280912E09E9
:1066B00081FFFEC102E000932F09809102028F5FEB
:1066C000809302028F71109130091295110F107E84
:1066D000182BE0903109D090320989E399E06FE7F7
:1066E00079E00E942230F8E0FF2EF092AC03109285
:1066F000AD038EEA93E064EF7CE049E050E00E9455
:1067000026098CE28093B10386E08093B7030E9450
:10671000D92FE092C403D092C5038BE08093C203CB
:106720001093C303E6ECF3E0DF011D92FA94E9F75E
:10673000809103028093C8038D5F8093030280E6FB
:106740008093CE030093CF0383E08093D003109215
:10675000D1031092D2031092D3031092D40310925B
:10676000D5030093D60384E08093D7030093D80326
:1067700086E28093D90382E36AE140E250E022E0BE
:106780000E946D2F8AE390E0AEC08091BE038F3EE1
:1067900079F48091BF038F3F59F48091C0038F3FFC
:1067A00039F48091C1038A3F19F42AE230E082C1B2
:1067B000C932D10508F47CC11091AC03183009F03E
:1067C00082C18091AD03863009F07DC186EC93E0F3
:1067D0006BE679E044E050E00E942F09009709F051
:1067E00072C18091B503813029F586EA93E00E9459
:1067F00011301092B40382E08093B50380EC93E0F3
:1068000066EB73E00E94D65086EB93E065E679E094
:106810000E94D65086EC93E06CEB73E00E94DE5051
:106820008CEB93E06BE679E00E94DE508AE290E028
:106830000E94692E80912E0983FF3AC11091B50301
:10684000123009F035C18CEB93E063E779E044E066
:1068500050E00E942F09009709F02AC189E399E0CE
:1068600066EB73E00E94D65010932E0921C11830B8
:1068700009F01EC18091AD03882309F019C18091F0
:10688000AE03853409F014C18EEB93E06BE679E03A
:1068900044E050E00E942F09009709F009C180915F
:1068A000B703813019F58091C2038830F9F4E09183
:1068B0003309F0913409309719F08AEB93E0099588
:1068C0000E9481301092C2038091C403883F28F057
:1068D0008091C5038F5F8093C5038091C403885F57
:1068E0008093C403CE010E94692EE2C00E945739F2
:1068F000882351F08091B703813131F4CE010E9499
:106900005C39882309F0D4C0C633D10528F48091BE
:10691000B703863009F0CCC08091C4038B3009F0F6
:10692000BEC08AEB93E06FE779E044E050E00E945C
:106930002F09009709F0BCC08091CF03382F82FF48
:1069400013C0E0913509F0913609309759F08091E4
:10695000C50382958695877063E040E050E020E0B3
:1069600030E0099585E090C09091B00380E02091DF
:10697000B103022F10E0082B192B8091CE03482F72
:1069800050E0E4E055954795EA95E1F7CA01880F94
:10699000991F880F991F081B190B0451104017FFEE
:1069A00002C000E010E080912F09823079F531FFBC
:1069B00021C034FF1FC080E090E060E00E940831F9
:1069C00088E18093CF03E0913709F091380930973F
:1069D00019F420E030E007C08091C30382958695CA
:1069E000877009959C0183E080932F09C9010E945B
:1069F000A9305EC081E080932F0934FF03C080E09E
:106A000090E002C0C801019664E046C0833081F581
:106A10000115110579F1E0913509F09136093097AA
:106A200049F1440F551F440F551FCE0108974E5D85
:106A30005F4F8417950708F4AC01C801840F951FB8
:106A4000C817D90710F0980103C09E01241B350B0D
:106A50008091C50382958695877060E00995809145
:106A60008409882319F0C80168E016C0C80108C06D
:106A70008530F1F030FF0BC08330D1F0C8010196B2
:106A800069E00E94083186E080932F0911C001154A
:106A9000110571F0C80160E00E94083109C08091C1
:106AA000040290910502BE010E9485319C0102C042
:106AB00020E030E0C901DF91CF911F910F91FF904D
:106AC000EF90DF900895CA32D10508F0D0CEF0CF14
:106AD000BC018091B7038130A1F48091C203882367
:106AE00081F48091CA03823461F48AEB93E044E03C
:106AF00050E00E942F099C0180E0232B19F481E0D3
:106B0000089580E008950F931F93CF93DF939C0126
:106B1000EB018A0110928309009729F08BE699E036
:106B2000B9010E94DE50209719F0CE010E94A030DA
:106B30000115110529F08BE799E0B8010E94DE509C
:106B400081E0DF91CF911F910F910895AF92BF9295
:106B5000CF92DF92FF920F931F93CF93DF938C011D
:106B6000EB01F42E1092830938E341E050E060E03D
:106B700070E018C0832F90E0FC01B3E0F595E79535
:106B8000BA95E1F7EB5BF64F877090705A016B0195
:106B900004C0AA0CBB1CCC1CDD1C8A95D2F720813A
:106BA0002A292083315031F785E699E0BE010E9401
:106BB000D650C80165E679E04F2D0E94C52EDF91C1
:106BC000CF911F910F91FF90DF90CF90BF90AF902A
:106BD0000895CF92DF92EF92FF920F931F93DF936E
:106BE000CF93CDB7DEB7EB84FC84CD84DE84DE01A9
:106BF0001F9601C0D801F6018491882309F4BCC016
:106C00000894C11CD11C843209F099C0F601089483
:106C1000C11CD11C8491863409F45FC0873434F4DC
:106C2000843469F0853409F08AC06EC08C34C9F1AF
:106C3000833509F445C0883409F081C00DC08D0149
:106C40000E5F1F4FF701668177818D919C914AE01D
:106C500050E00E94E5097EC02C91822F992787FD84
:106C6000909514E0959587951A95E1F78F702F70A0
:106C70002A300CF0295F8A300CF0895F8D010E5F9D
:106C80001F4FF701A681B781805DFD018193205DD3
:106C900011962C933196D7011796FC93EE93169785
:106CA000A9CF8D010C5F1F4F6D917D918D919C91AE
:106CB000F701468157812AE030E00E94230A4AC04A
:106CC0008D010E5F1F4F6D917C91D70116968D91AE
:106CD0009C9117970E944C093DC08D010E5F1F4F7C
:106CE0002D913C910AC0D7011696ED91FC91179712
:106CF00081931796FC93EE931697F9012F5F3F4F00
:106D00008491882381F776CF8D010E5F1F4F2D91DF
:106D10003C910AC0D7011696ED91FC91179781938B
:106D20001796FC93EE931697F999FECF32BD21BDCD
:106D3000F89A80B52F5F3F4F882361F75BCFF7014B
:106D400026813781F90181939F01F70137832683DB
:106D50008D0150CFD70116968D919C911797FC010C
:106D600001900020E9F73197E81BF90B8E0F9F1F68
:106D7000F701978386833ECFCF91DF911F910F91CB
:106D8000FF90EF90DF90CF900895DF93CF9300D0E6
:106D900000D000D0CDB7DEB7DE011196E4E4F3E019
:106DA00086E001900D928150E1F786E191E0E0EA02
:106DB000F3E0DF019C011D9221503040E1F780910A
:106DC0008509833019F467E779E003C0BE016F5F7E
:106DD0007F4F84E490E043E450E00E943A30809199
:106DE0008509833039F080EA93E0BE016F5F7F4F01
:106DF0000E94D65081E08093CA038093CB0386E043
:106E00008093CC038091920990919309A091940969
:106E1000B09195098093CE039093CF03A093D003B4
:106E2000B093D10380918509833039F48AEC93E0E3
:106E30000C966BE679E00E94DE5086EE93E065E604
:106E400079E00E94D650A6EBB4E0EDE1F2E002C09A
:106E500081918D9332E0E332F307D1F79091850968
:106E6000992311F083E001C081E08093BC048DE39D
:106E70008093BD0487E08093BE0481E08093BF04CB
:106E8000A0ECB4E0E5E6F9E002C081918D9389E0E1
:106E9000EB36F807D1F78CE08093C60480E180934D
:106EA000C704E6E0F2E0A8ECB4E002C081918D9363
:106EB00022E0E631F207D1F728ED34E0309397096C
:106EC00020939609913069F582E38093D80484E099
:106ED0008093D904D9011296EBE6F9E002C08191C2
:106EE0008D9339E0EF36F307D1F786E38093DE0424
:106EF00084E08093DF0480EE94E090939709809380
:106F00009609DC01E7E7F9E002C081918D9389E001
:106F1000EB37F807D1F784EE94E0909397098093CC
:106F200096092091960930919709D901E7E1F2E09D
:106F300002C081918D9382E0ED31F807D1F7C9014C
:106F4000069690939709809396098A5C93400E94D5
:106F5000273226960FB6F894DEBF0FBECDBFCF9175
:106F6000DF910895DF92EF92FF920F931F93CF93DB
:106F7000DF938C0180918509823009F4F7C083305A
:106F800030F4882351F1813009F054C14AC0833074
:106F900021F0843009F04EC1E9C00E94C956209109
:106FA0008A0930918B0940918C0950918D09E090AC
:106FB0008609F090870900918809109189092E0DA2
:106FC0003F1D401F511F621773078407950708F480
:106FD00031C10E94C53684E017C00E94C956609333
:106FE0009209709393098093940990939509109254
:106FF0006B0910926C0910926D0910926E090E9433
:10700000C5360E94702D81E0809385090E94C95683
:1070100060938E0970938F098093900990939109E2
:1070200009C10634110508F4F0C08091C30383340C
:1070300009F0EBC02091CE033091CF034091D003F3
:107040005091D1038091920990919309A091940954
:10705000B0919509281739074A075B0709F0D5C091
:10706000CAEBD4E0FE01A80140565C4FDF01119647
:1070700091819D012F5F3F4F8081853321F41196CF
:107080008C91823039F0F901E90FF11DE417F50711
:1070900068F3BBC08BE699E06AED73E00E94DE50B6
:1070A00050EAE52E53E0F52EE00EF11EFE0131967A
:1070B000D9808F010F5F1F4F88818630A9F08730FC
:1070C00030F4813059F0833009F045C00AC086336E
:1070D000E9F18A3361F08333F1F509C08FE699E075
:1070E00037C083E799E034C08BE799E031C0618114
:1070F00070E080E090E0982F872F762F6627F801C8
:107100002181620F711D811D911D982F872F762F70
:1071100066272281620F711D811D911D982F872F77
:10712000762F66272381620F711D811D911D28EE28
:1071300033E040E050E00E94475C60938A0970931E
:107140008B0980938C0990938D0905C087E799E09E
:10715000B8010E94DE50E801CD0DD11DCE15DF052E
:1071600008F4A4CF0E94C53682E04ECF0634110544
:1071700008F44BC08091C303833409F046C02091CA
:10718000CE033091CF034091D0035091D103809131
:10719000920990919309A0919409B09195092817AB
:1071A00039074A075B0789F5EAEBF4E0A801405686
:1071B0005C4FDF01119691819D012F5F3F4F8081D0
:1071C000853321F411968C91853039F0F901E90F5E
:1071D000F11DE417F50768F318C00E946B2D0E949B
:1071E000C9566093860970938709809388099093A4
:1071F000890980917309882321F083E799E00E942F
:10720000A03083E08093850915C00E94C956209163
:107210008E0930918F094091900950919109205F1A
:10722000384D4F4F5F4F261737074807590710F45F
:1072300010928509DF91CF911F910F91FF90EF90F0
:10724000DF900895CF93DF9381E08093830990913D
:107250006A09892F82958F70805D809314029F70D8
:10726000905D90931502109285090E94C956EB011A
:1072700004C00E94E02D0E94B237809185098330BE
:1072800061F00E94C9566C1B7D0B60567A4E28F443
:107290000E94A12D882389F3ECCF90E0809185098D
:1072A000833009F491E0892FDF91CF910895809187
:1072B000C009811181E00895CF92DF92EF92FF9291
:1072C0000F931F93CF93DF93C8E9D9E030E0CC242C
:1072D000DD2429C02A814B818091C40390E0042FD2
:1072E00010E080179107D9F49091C5039217B9F473
:1072F0008C818823A1F02091C70330E028503040D2
:10730000F090C603EE242E0D3F1DE881F981892FF0
:10731000942F6AEB73E04AEC53E0099531E008944E
:10732000C11CD11C25968091C00990E0C816D906D1
:107330008CF2832FDF91CF911F910F91FF90EF90EF
:10734000DF90CF900895FC01EF5BFD4F10827796A0
:107350001082089510921C0C0895FC01E55AFD4F0F
:107360008081882319F4862F0E94EA500895EF92B5
:10737000FF920F931F937C018B01472F5527FC0130
:10738000858D968D480F591F60E070E0C7018F5BB7
:107390009F4F0E9488511070000F111F0E0D1F1D6E
:1073A0000E5B1F4FF801308120E08291280F311DC4
:1073B000C9011F910F91FF90EF9008958F929F92B6
:1073C000AF92BF92CF92DF92EF92FF920F931F93F3
:1073D000CF93DF93EC01C85ADD4F8881C855D24066
:1073E000813009F0C4C0CC5ADD4FE880F9800A81B1
:1073F0001B81C455D240E114F1040105110559F473
:10740000C25BDD4F88819981CE54D240892B19F41B
:107410006DEF7FEFB3C0298530E040E050E0C80158
:10742000B7010E94995C611571058105910589F488
:10743000E114F1040105110561F08E01025B1D4F9D
:10744000F80160817181CE010E94B739F801918302
:107450008083A984BB24CC24DD24EA84FB8400E05F
:1074600010E08D899E89AF89B88DE80EF91E0A1F3C
:107470001B1F6B897C8980E090E02C8530E040E028
:1074800050E00E94475CE60EF71E081F191FF4E546
:107490008F2EF2E09F2E8C0E9D1EF4016081718173
:1074A00082819381A60195010E94995CE60EF71EE8
:1074B000081F191F8D859E85A0E0B0E0E4E0B69519
:1074C000A79597958795EA95D1F7E80EF91E0A1FBB
:1074D0001B1FC25BDD4F68817981CE54D24080E0B2
:1074E00090E06250704080409040A60195010E945B
:1074F000475CE60EF71E081F191FCE018F5B9F4FDA
:10750000B801A7010E948851882319F0682F70E004
:1075100035C0F4012081318142815381DA01C901F2
:107520000196A11DB11D80839183A283B383C05BAB
:10753000DD4FE880F9800A811B8179E0880F991F6F
:10754000AA1FBB1F7A95D1F7E816F9060A071B0791
:1075500018F060E072E012C069E0220F331F441F90
:10756000551F6A95D1F7B701621B730B07C08823BB
:1075700019F061EF7FEF02C060EF7FEFCB01DF9189
:10758000CF911F910F91FF90EF90DF90CF90BF9020
:10759000AF909F908F9008954F925F926F927F92DD
:1075A0008F929F92AF92BF92CF92DF92EF92FF9213
:1075B0000F931F93CF93DF934C013B018DE390E03A
:1075C000880E991EE401E880F9800A811B81E3ECB2
:1075D000FFEF8E0E9F1E49E5442E42E0542E480CCC
:1075E000591CE2018881998135E0880F991F3A95ED
:1075F000E1F7AC01452F5527469520E03EEF429F2D
:10760000E001439FD00D529FD00D1124C80FD91F08
:107610005A01CC24DD24AE0CBF1CC01ED11E840137
:107620000F5B1F4FC801B601A5010E94885117C00A
:10763000A096F20180819181019691838083F2E08E
:10764000C030DF0761F40894A11CB11CC11CD11C1F
:10765000C801B601A5010E948851C0E0D0E0F40144
:10766000EC0FFD1FEF5BFF4F8081882309F49DC065
:10767000DE011B96F401EA0FFB1FEF5BFF4F8081D9
:107680008871B1F6F401EC0FFD1FEF5BFF4F8081B5
:10769000853E71F2CF5BDF4FA4014C0F5D1FC154DB
:1076A000D04020E030E0B301620F731FFA018191F6
:1076B000AF01FB0180832F5F3F4F2830310599F7E1
:1076C0002896F401EC0FFD1F9E0128503040EF5B1F
:1076D000FF4F8191E301898781918A8780818B8720
:1076E00018861C86A80DB91DAF5BBF4F8C918D8786
:1076F000280D391D205B3F4FF901908180E0E901A1
:107700004A919E01840F911DF301978786872D5F13
:107710003F4FE901988180E0F90142919F01840F78
:10772000911DE301998B888B255F3F4FF901908173
:1077300080E0E9014A919E01840F911DF301938B32
:10774000828B2B5F3F4FE901488150E060E070E0A1
:10775000742F662755274427F901829190E0A0E015
:10776000B0E0DC0199278827482B592B6A2B7B2B0B
:10777000EF019A9180E0FE01229130E0822B932B61
:10778000A0E0B0E0482B592B6A2B7B2BF301448BF4
:10779000558B668B778BF401E75AFD4F8081918181
:1077A00001969183808380E001C081E0DF91CF91D9
:1077B0001F910F91FF90EF90DF90CF90BF90AF900F
:1077C0009F908F907F906F905F904F9008956F92F1
:1077D0007F928F929F92AF92BF92CF92DF92EF9261
:1077E000FF920F931F93CF93DF93EC016B01ED9604
:1077F000E880F9800A811B81ED9789E5A82E82E057
:10780000B82EAC0EBD1ED5011D921C92B1E48B2E7C
:10781000912C8C0E9D1EC401B801A7010E948851B5
:10782000F4018081882309F4D8C020E030E022C030
:10783000205E3F4FD5018D919C91119701968D93BC
:107840009C93B2E020303B0761F40894E11CF11CEA
:10785000011D111DC401B801A7010E94885120E03B
:1078600030E0FE01E20FF31FEF5BFF4F80818823C2
:1078700009F4B3C0ABE06A2E712C620E731EFE01D8
:10788000E60DF71DEF5BFF4F8081887189F6FE01E1
:10789000E20FF31FEF5BFF4F8081853E49F22F5BC4
:1078A0003F4FBE01620F731F2154304040E050E053
:1078B0008601040F151FFB018191BF01D8018C9334
:1078C0004F5F5F4F4830510599F7285F3F4FFE01EA
:1078D000E20FF31F28503040EF5BFF4F8191D6013C
:1078E00019968C93199781911A968C931A97808187
:1078F0001B968C931B9718961C9218971C961C929B
:107900006C0E7D1EE1E4F0E06E0E7F1ED3018C91C3
:10791000F60185872C0F3D1F205B3F4FD9019C91BD
:1079200080E0F90142919F01840F911DD6011F96BD
:107930009C938E931E972D5F3F4FF901908180E0BD
:10794000D9014E919D01840F911DF601918B808B81
:10795000255F3F4FD9019C9180E0F90142919F0141
:10796000840F911DD60153969C938E9352972B5F53
:107970003F4FF901408150E060E070E0742F6627CE
:1079800055274427D9018E919D0190E0A0E0B0E0F9
:10799000DC0199278827482B592B6A2B7B2BF9016F
:1079A000929180E0229130E0822B932BA0E0B0E016
:1079B000482B592B6A2B7B2BD60154964D935D9304
:1079C0006D937C935797FE01E75AFD4F808191811B
:1079D00001969183808380E001C081E0DF91CF91A7
:1079E0001F910F91FF90EF90DF90CF90BF90AF90DD
:1079F0009F908F907F906F9008956F927F928F925B
:107A00009F92AF92BF92CF92DF92EF92FF920F932D
:107A10001F93DF93CF93CDB7DEB7A5970FB6F8943A
:107A2000DEBF0FBECDBF7C016B01AB0120E030E0BB
:107A30000CC0FA019081892F81568A3108F4905246
:107A4000FA019193AF012F5F3F4FF60101900020A3
:107A5000E9F73197EC19FD092E173F0750F38E0116
:107A6000025F1F4FC701B8010E94E73BF82EF1E00B
:107A70008F1709F490C040E050E0B8019E012F5FDD
:107A80003F4F06C0F901E40FF51F80834F5F5F4F42
:107A9000FB01E40FF51F8081803219F04830510559
:107AA00089F7CE010196FC01E40FF51F2EE2208339
:107AB000DA01119647E1642E712C6C0E7D1E8A0F3F
:107AC0009B1FB301AE01455E5F4F04C0FC012193D3
:107AD000CF011196FB012081203229F06F5F7F4F8B
:107AE0006417750799F78E010F5F1F4FA00FB11F25
:107AF0001C92C801B6010E9443090097E9F54DC0E8
:107B000081EC99E0B5010E94CC3AF82E882309F067
:107B10003FC080E090E005C0F801E80FF91F208326
:107B20000196F501E80FF91F2081203219F0883005
:107B3000910591F7F801E80FF91FE082DC01119639
:107B4000C8018A0F9B1FA30104C0FC012193CF0130
:107B50001196FA012081203229F04F5F5F4F4815BE
:107B6000590599F7A00FB11F1C92C801B6010E94D8
:107B70004309009729F611C03EE0A32EB12CAC0EAC
:107B8000BD1E2EE2E22E9BE1892E912C8C0E9D1EB5
:107B9000FF2009F4B5CF80E001C081E0A5960FB6C3
:107BA000F894DEBF0FBECDBFCF91DF911F910F9133
:107BB000FF90EF90DF90CF90BF90AF909F908F900D
:107BC0007F906F9008953F924F925F926F927F9255
:107BD0008F929F92AF92BF92CF92DF92EF92FF92DD
:107BE0000F931F93DF93CF93CDB7DEB7A5970FB653
:107BF000F894DEBF0FBECDBF8C01B62EC72E342E3B
:107C00000F5B1D4FF801808101541240882311F051
:107C100081E1EFC0862F972F9C01A90120E030E081
:107C20000CC0FA019081892F81568A3108F4905254
:107C3000FA019193AF012F5F3F4FAB2DBC2DFD019A
:107C400001900020E9F73197EA1BFB0B2E173F0745
:107C500040F33EE0E32EF12CEC0EFD1EC801B7010F
:107C60000E94E73BD82EF1E08F1709F4C1C040E035
:107C700050E0B7019E012F5F3F4F06C0F901E40FAE
:107C8000F51F80834F5F5F4FFB01E40FF51F80817D
:107C9000803219F04830510589F7CE010196FC0178
:107CA000E40FF51F2EE22083DA01119627E1422E20
:107CB000512C4C0E5D1E8A0F9B1FB201AE01455E1A
:107CC0005F4F04C0FC012193CF011196FB0120817D
:107CD000203229F06F5F7F4F6417750799F77E0197
:107CE0000894E11CF11CAE0DBF1D1C92C7016B2D49
:107CF0007C2D0E944309009709F06BC0F701D80161
:107D0000AF5BBD4F9E01225F3F4F81918D93E21784
:107D1000F307D9F748C081EC99E0B4010E94CC3A4E
:107D2000D82E882309F061C080E090E005C0F701FB
:107D3000E80FF91F20830196F401E80FF91F208155
:107D4000203219F08830910591F7F701E80FF91FFB
:107D5000A082DC011196C7018A0F9B1FA20104C0FB
:107D6000FC012193CF011196FA012081203229F0E4
:107D70004F5F5F4F4615570599F7AE0DBF1D1C921B
:107D8000C7016B2D7C2D0E944309009721F6F70156
:107D9000D801AF5BBD4F9E01225F3F4F81918D9314
:107DA000E217F307D9F7025B1D4F88A199A1F801EB
:107DB000819391938AA19BA1ACA1BDA18193919341
:107DC000A193B1931192119211921192308280E09D
:107DD00010C0AEE08A2E912C8C0E9D1EFEE2AF2EBE
:107DE000EBE16E2E712C6C0E7D1EDD2009F493CF1D
:107DF00080E1A5960FB6F894DEBF0FBECDBFCF9140
:107E0000DF911F910F91FF90EF90DF90CF90BF9087
:107E1000AF909F908F907F906F905F904F903F902A
:107E200008950F931F93CF93DF93EC01862F0E9449
:107E3000F0518E010F5B1F4FC80140E050E060E041
:107E400070E00E948851882311F080EF84C1C15CEA
:107E5000DD4F8881CF53D240853509F079C1C05CB0
:107E6000DD4F8881C054D2408A3A09F071C1CD5F9C
:107E7000DD4F7881C350D2407883C65FDD4F2881C3
:107E800030E040E050E0522F4427332722278A91E8
:107E900090E0A0E0B0E0DC0199278827280F391F87
:107EA0004A1F5B1F9A9180E06A91C750D240860FAB
:107EB000911DA0E0B0E0280F391F4A1F5B1F2983E6
:107EC0003A834B835C83C25FDD4F288130E040E022
:107ED00050E0522F4427332722278A9190E0A0E0D8
:107EE000B0E0DC0199278827280F391F4A1F5B1F44
:107EF0009A9180E06A91CB50D240860F911DA0E00C
:107F0000B0E0280F391F4A1F5B1F2D833E834F832C
:107F10005887743031F0763021F0763811F082EFE6
:107F20001AC149815A816B817C81C8010E948851A4
:107F3000882311F080EE0FC1C15CDD4F8881CF53E3
:107F4000D240853509F006C1C05CDD4F8881C05440
:107F5000D2408A3A09F0FEC0C25BDF4F8881CE541E
:107F6000D0408987C05BDF4F988180E02A91CF5451
:107F7000D040820F911D9B878A87CF5ADF4F88811F
:107F8000C155D0408C87CD5ADF4F988180E02A912F
:107F9000C255D040820F911D9E878D87CB5ADF4FEF
:107FA000988180E02A91C455D040820F911DA0E0B5
:107FB000B0E08F87988BA98BBA8B0097A105B1058C
:107FC00031F5CC59DF4F288130E040E050E0522FAE
:107FD0004427332722278A9190E0A0E0B0E0DC011B
:107FE00099278827280F391F4A1F5B1F9A9180E025
:107FF0006A91C156D040860F911DA0E0B0E0280FD5
:10800000391F4A1F5B1F2F87388B498B5A8BC85AE1
:10801000DF4F788160E08A91C755D040680F711DAD
:108020007C8B6B8BC05ADF4F288130E040E050E002
:10803000522F4427332722278A9190E0A0E0B0E016
:10804000DC0199278827280F391F4A1F5B1F9A9147
:1080500080E0EA91CD55D0408E0F911DA0E0B0E0B8
:10806000280F391F4A1F5B1F2D8B3E8B4F8B588F5C
:10807000C559DF4F288130E040E050E0522F4427BF
:10808000332722278A9190E0A0E0B0E0DC01992715
:108090008827280F391F4A1F5B1F9A9180E0EA91B9
:1080A000C856D0408E0F911DA0E0B0E0280F391FB8
:1080B0004A1F5B1F298F3A8F4B8F5C8FEA85FB85A8
:1080C0009F0140E050E089819A81AB81BC81280FFB
:1080D000391F4A1F5B1F8C8590E0DC01A69FC00101
:1080E000A79F900DB69F900D1124A0E0B0E0280F3F
:1080F000391F4A1F5B1FED96288339834A835B83B0
:10810000ED9789819A818E0F9F1F9E8F8D8F860F8D
:10811000971F98A38F8F6D817E818F81988549E00D
:10812000660F771F881F991F4A95D1F70E94565BEB
:1081300020E030E040E855E30E94E45B69A37AA3C5
:108140008BA39CA3C55ADD4F81E0888380E003C0E8
:1081500081EF01C081EEDF91CF911F910F910895C2
:108160000F931F938C01FC01868160E00E94CB5726
:1081700081E090E00E944757F801868161E00E940B
:10818000CB5781E090E00E944757F801868160E07C
:108190000E94CB5784E690E00E9447571F910F91B1
:1081A0000895CF92DF92EF92FF920F931F93CF9398
:1081B000DF93D82EC92E282F392FC9018C01C0E09A
:1081C000D0E0E62EFF24F801878161E00E948C5701
:1081D000B7010C2E02C0759567950A94E2F761709D
:1081E000F80187810E94CB5721960F5F1F4FC8303F
:1081F000D10549F78D2D9C2D0E94B040DF91CF9184
:108200001F910F91FF90EF90DF90CF900895CF9244
:10821000DF92EF92FF920F931F93CF93DF93D82EAD
:10822000C92E282F392FC9018C01C0E0D0E0E62EDD
:10823000FF24F801878161E00E948C57B7010C2E62
:1082400002C0759567950A94E2F76170F80187811D
:108250000E94CB5721960F5F1F4FC430D10549F7BD
:108260008D2D9C2D0E94B040DF91CF911F910F91D9
:10827000FF90EF90DF90CF9008951F93CF93DF93FF
:10828000EC01162F8C81642F0E94CB578D818F3F7C
:1082900019F060E00E94CB578F8584FF05C0CE01A6
:1082A000612F0E94D1400EC0612F70E084E075956F
:1082B00067958A95E1F7CE010E940741CE01612FB3
:1082C0000E940741DF91CF911F91089541E00E94E4
:1082D0003D4181E090E0089540E00E943D410895D5
:1082E000EF92FF920F931F93CF93DF938C017A014C
:1082F0006770660F660F660F60640E946C41C0E095
:10830000D0E0D801ED91FC91D701AC0FBD1F0190D9
:10831000F081E02DC8016C9109952196C830D105F6
:1083200081F7DF91CF911F910F91FF90EF9008950A
:10833000FC016089862F8160808B6960CF010E947B
:108340006C410895FC0160896E7F608B68600E94BB
:108350006C410895FC016089862F8460808B6C607D
:10836000CF010E946C410895DF93CF93CDB7DEB764
:1083700028970FB6F894DEBF0FBECDBF9C01FE015B
:108380003196A2E5B3E088E00D9001928150E1F7CB
:10839000F9018389481710F0482F4150E42FF0E08D
:1083A000EE0FFF1FEC0FFD1F8181680F6068C90190
:1083B0000E946C4128960FB6F894DEBF0FBECDBF69
:1083C000CF91DF91089561E00E946C4180ED97E0CC
:1083D0000E9447570895CF93DF93EC01423018F085
:1083E0008F8588608F874B8B1C8A222329F0413030
:1083F00019F48F8584608F8780E593EC0E9447573E
:108400008C8160E00E94CB578E8160E00E94CB5748
:108410008D818F3F19F060E00E94CB576F8564FD1E
:108420001DC0CE0163E00E94074184E991E10E94F2
:108430004757CE0163E00E94074184E991E10E9421
:108440004757CE0163E00E94074186E990E00E9411
:108450004757CE0162E00E94074116C06062CE011C
:108460000E946C4184E991E10E9447576F856062E8
:10847000CE010E946C4186E990E00E9447576F85CB
:108480006062CE010E946C416F856062CE010E94E5
:108490006C4184E0888BCE010E94AA41CE010E94EB
:1084A000E34182E0898BCE0166E00E946C41DF915E
:1084B000CF9108956F927F928F92AF92CF92EF9269
:1084C0000F931F93DF93CF93CDB7DEB73C01162FE9
:1084D000842FF301448325830683E782C086A18627
:1084E00082869D8593879E8594879F8595879889A9
:1084F000968761E00E948C57F30185818F3F19F0C8
:1085000061E00E948C57F301868161E00E948C57E4
:10851000112319F0F301178603C080E1F301878767
:10852000C30160E141E020E00E94EB41CF91DF9187
:108530001F910F91EF90CF90AF908F907F906F90A1
:1085400008958F929F92AF92BF92CF92DF92EF9257
:10855000FF920F931F93CF93DF937B018C01EA016E
:108560002CE330E040E050E00E94995C6883C80151
:10857000B7012CE330E040E050E00E94995C122FFC
:10858000032FF42EE52E622F732F842F952F2CE3CB
:1085900030E040E050E00E94995C6983612F702FC9
:1085A0008F2D9E2D2CE330E040E050E00E94995C3E
:1085B000122F032FF42EE52E622F732F842F952F69
:1085C00028E130E040E050E00E94995C6A83612F2E
:1085D000702F8F2D9E2D28E130E040E050E00E946A
:1085E000995C79018A01C801B7016C5F7F4F8F4F99
:1085F0009F4F27E030E040E050E00E94995C6F5FC1
:108600006B8320E0AA24BB24650101C02F5F822E6A
:108610009924F401EE54F84FCF0183709070892BA8
:1086200099F4CF0164E670E00E94865C892B39F4EE
:10863000CF0160E971E00E94865C892B29F48EE607
:1086400091E0A0E0B0E004C08DE691E0A0E0B0E0F1
:10865000A80EB91ECA1EDB1EC501A0E0B0E0E816D8
:10866000F9060A071B0790F62E83F401EE54F84F23
:1086700083E0882E912C8E229F228114910499F4FC
:10868000CF0164E670E00E94865C892B39F4CF014B
:1086900060E971E00E94865C892B29F48EE691E006
:1086A000A0E0B0E004C08DE691E0A0E0B0E0A81A40
:1086B000B90ACA0ADB0A980187010A191B092C09A1
:1086C0003D09CF0164E670E00E94865C7C01CF0129
:1086D00060E971E00E94865CAC01EAE5F3E060E0ED
:1086E000613051F48114910449F4E114F10441F42E
:1086F0004115510529F002C0808103C08CE101C001
:108700008DE190E0A0E0B0E0081719072A073B07C9
:1087100040F0081B190B2A0B3B0B6F5F31966C3036
:10872000F9F66F5F6D83802F8F5F8C83DF91CF9120
:108730001F910F91FF90EF90DF90CF90BF90AF907F
:108740009F908F900895EF92FF920F931F937B015C
:108750008C018091340C9091350CA091360CB09125
:10876000370CE816F9060A071B0771F0C801B701B4
:1087700049E25CE00E94A142E092340CF092350C98
:108780000093360C1093370C1F910F91FF90EF90D0
:1087900008950E94A34320912F0C30E02E54384FAF
:1087A000C90108950E94A34380912E0C90E0089582
:1087B0000E94A34380912C0C90E008950E94A34353
:1087C00080912D0C90E008950E94A34380912A0C83
:1087D00090E008950E94A34380912B0C90E00895AF
:1087E0004F925F926F927F928F929F92AF92BF92C1
:1087F000CF92DF92EF92FF920F931F93CF93DF936D
:108800004C01DC0116961C91612F70E080E090E035
:1088100020E833E341EE51E00E94475C5B016C01CC
:1088200022EB37E0E12FF0E0EE54F84F1DC0C90114
:1088300083709070892BB1F4C90164E670E00E94E6
:10884000865C892B39F4C90160E971E00E94865C7D
:10885000892B41F480E891E5A1E0B0E0A80EB91EB3
:10886000CA1EDB1E2F5F3F4F2E173F0701F7D401B3
:1088700015968C91482E5524C90164E670E00E943B
:10888000865C7C01C90160E971E00E94865C8C0114
:10889000C1E0D0E093E0692E712C6222732227C0E0
:1088A000C230D10591F46114710479F4E114F1043A
:1088B00019F40115110549F480E89BE3A6E2B0E044
:1088C000A80EB91ECA1EDB1E11C0FE01E75AFC4FDE
:1088D000608170E080E090E020E831E541E050E028
:1088E0000E94475CA60EB71EC81ED91E2196C4154D
:1088F000D505B4F2D40112966C9170E080E090E05E
:1089000020E13EE040E050E00E94475C7B018C01AA
:10891000F401618170E080E090E02CE330E040E021
:1089200050E00E94475CE60EF71E081F191FD40195
:108930008C91E80EF11C011D111D14966C9170E0D4
:1089400061507040882777FD8095982F20E831E5A9
:1089500041E050E00E94475CE60EF71E081F191F19
:10896000EA0CFB1C0C1D1D1DB701C801DF91CF9146
:108970001F910F91FF90EF90DF90CF90BF90AF903D
:108980009F908F907F906F905F904F90089560932D
:108990002302709324028093250290932602089567
:1089A00060931F0C7093200C8093210C9093220CE9
:1089B00020912302309124024091250250912602F9
:1089C000260F371F481F591F2093230C3093240C68
:1089D0004093250C5093260C82E090E09093280C55
:1089E0008093270C0E94C9566093300C7093310C11
:1089F0008093320C9093330C0895EF92FF920F9373
:108A00001F931CC02F5F3F4F4F4F5F4F20931F0C92
:108A10003093200C4093210C5093220C88EE93E06D
:108A2000A0E0B0E0E80EF91E0A1F1B1FE092300C18
:108A3000F092310C0093320C1093330C0E94C95603
:108A4000E090300CF090310C0091320C1091330C0E
:108A50006E197F09800B910B20911F0C3091200C17
:108A60004091210C5091220C685E734080409040F0
:108A700048F68091230C9091240CA091250CB09184
:108A8000260C281739074A075B07E8F0E0911D0C10
:108A9000F0911E0C3097B9F00995611571058105AB
:108AA000910519F00E94D0440EC020E030E0809182
:108AB000270C9091280C892B11F021E030E03093A5
:108AC000280C2093270C60911F0C7091200C809132
:108AD000210C9091220C1F910F91FF90EF9008951F
:108AE00090931E0C80931D0C80911F0C9091200C74
:108AF000A091210CB091220C8093230C9093240C14
:108B0000A093250CB093260C0E94FD440895482F95
:108B10006AE00E94665C282F30E084E0220F331F59
:108B20008A95E1F7842F0E94665C892F820F089551
:108B3000CF93DF93EC018091380C9091390C8836FB
:108B4000910559F585EC9CE068E670E00E9434538D
:108B500085EC9CE060E00E94B65388810E948745C6
:108B6000682F70E06F77707085EC9CE00E94B653C0
:108B700089810E948745682F85EC9CE00E94B6534E
:108B80008A810E948745682F85EC9CE00E94B6533D
:108B90008B810E948745682F2DC08F36910509F083
:108BA0004AC085EC9CE06FE670E00E94345385EC8F
:108BB0009CE060E00E94B65388810E948745682F40
:108BC000606885EC9CE00E94B65389810E948745CD
:108BD000682F85EC9CE00E94B6538A810E948745ED
:108BE000682F85EC9CE00E94B6538B810E948745DC
:108BF000682F686085EC9CE00E94B6538C810E94CF
:108C00008745682F85EC9CE00E94B6538D810E94B9
:108C10008745682F85EC9CE00E94B6538E818E516B
:108C20000E948745682F85EC9CE00E94B65385EC36
:108C30009CE00E94F953DF91CF91089588E690E07F
:108C40009093390C8093380C85EC9CE068E670E0DA
:108C50000E94345385EC9CE060E00E94B65385ECA2
:108C60009CE00E94F9538823D9F08FE690E090931E
:108C7000390C8093380C85EC9CE06FE670E00E9424
:108C8000345385EC9CE060E00E94B65385EC9CE098
:108C90000E94F953882321F01092390C1092380C5D
:108CA00008951F93CF93DF93EC016091380C70917E
:108CB000390C6115710509F46FC085EC9CE00E94C8
:108CC000345385EC9CE060E00E94B65385EC9CE058
:108CD0000E94F9536091380C7091390C85EC9CE03E
:108CE00047E050E00E940A5485EC9CE00E94475304
:108CF000282F2F7722952F701AE0219F90011124A1
:108D00008F70820F888385EC9CE00E944753282F48
:108D100022952F70219F900111248F70820F8983DB
:108D200085EC9CE00E944753282F2F7322952F70CB
:108D3000219F900111248F70820F8A8385EC9CE023
:108D40000E94475387708B8385EC9CE00E944753B9
:108D5000282F22952F70219F900111248F70820F50
:108D60008C8385EC9CE00E944753282F22952F701E
:108D7000219F900111248F70820F8D8385EC9CE0E0
:108D80000E944753282F2F70225E82958F70819FFB
:108D9000C0011124280F2E83DF91CF911F910895D8
:108DA0000F931F93DF93CF93CDB7DEB727970FB6FF
:108DB000F894DEBF0FBECDBF8E010F5F1F4FA8011D
:108DC0000E94A142C8010E94984527960FB6F894C8
:108DD000DEBF0FBECDBFCF91DF911F910F910895E0
:108DE0000F931F93DF93CF93CDB7DEB727970FB6BF
:108DF000F894DEBF0FBECDBF8E010F5F1F4FC801BD
:108E00000E945146C8010E94F04327960FB6F8947D
:108E1000DEBF0FBECDBFCF91DF911F910F9108959F
:108E200085EC9CE00E940E5408959C01F999FECFB8
:108E300032BD21BDF89A80B508959C01F999FECF05
:108E40001FBA32BD21BD60BD0FB6F894FA9AF99AE7
:108E50000FBE0895E0916D0CF0916E0C0995089588
:108E6000DB01482F50E0405F5F4F84E0440F551F07
:108E70008A95E1F750961C92509720E030E0F999DE
:108E8000FECFC901840F951F92BD81BDF89A80B5B0
:108E9000FD01E20FF31F8083882331F02F3031056D
:108EA00019F02F5F3F4FEBCF0895DB01482F50E0C3
:108EB000405F5F4F94E0440F551F9A95E1F750963D
:108EC0001C92509720E030E0FD01E20FF31FE0819B
:108ED000F999FECF1FBAC901840F951F92BD81BDBC
:108EE000E0BD0FB6F894FA9AF99A0FBEEE2331F06E
:108EF0002F30310519F02F5F3F4FE6CF089586E6FA
:108F000094E0FC01E750F84FE081F999FECF1FBAD9
:108F100092BD81BDE0BD0FB6F894FA9AF99A0FBEE2
:108F2000019624E08C36920761F7089580E694E07C
:108F3000FC01E750F84FE081F999FECF1FBA92BDCE
:108F400081BDE0BD0FB6F894FA9AF99A0FBE01966A
:108F500024E08636920761F70895282F27708695BA
:108F60008695869590E0662369F0FC01ED5AF34FF3
:108F700081E090E002C0880F991F2A95E2F72081D6
:108F8000282B0DC0FC01ED5AF34F81E090E002C0A8
:108F9000880F991F2A95E2F7809520812823208346
:108FA00008951092530C1092540C1092550C10927C
:108FB000560C1092570C1092580C0895E7E2F2E00C
:108FC00020E030E0F999FECF32BD21BDF89A80B59E
:108FD00080832F5F3F4F37962332310599F7809179
:108FE00090028F5F8093510C90E023E0880F991FCF
:108FF0002A95E1F78093520C0895E5E1F3E082E2CF
:1090000090E02081F999FECF1FBA92BD81BD20BDAD
:109010000FB6F894FA9AF99A0FBE019737972FEF87
:109020008F3F920771F7809190028F5F8093510C70
:1090300090E033E0880F991F3A95E1F78093520C46
:109040000895AC01FB010FC0F999FECF1FBADA01F8
:10905000A80FB11DB2BDA1BD20BD0FB6F894FA9AFC
:10906000F99A0FBE31968E2F861B2081222361F73D
:10907000F999FECF1FBA480F511D52BD41BD10BC1A
:109080000FB6F894FA9AF99A0FBE0895582F282F20
:10909000392FF9018E2F851BF999FECF90E0805C66
:1090A0009F4F92BD81BDF89A80B59081882331F0A1
:1090B000992349F0891739F43196ECCF80E0992350
:1090C00019F481E0089580E0089510923D0C10920B
:1090D0003C0C8EE493E090933B0C80933A0C089503
:1090E000EF92FF920F931F93CF93DF93E82E162FEB
:1090F000042FF22E662321F0623081F4222371F0D6
:109100008E2D0E941F58892B11F000E024C0FF20F3
:1091100011F480E001C080E8082B1DC0C0E0D0E061
:109120008E2D0E941F58892B81F4113031F012309E
:1091300061F483E0C032D80744F461E070E080E07D
:1091400090E00E94D7562196EBCFFF2019F4C05231
:10915000D3400CF00068802FDF91CF911F910F91C9
:10916000FF90EF9008950F931F93082F10916F0CAD
:10917000107861E070E080E090E00E94D7568FE1C7
:109180000E941F58892B21F48FE1602F41E013C00A
:109190008EE10E941F58892B21F48EE1602F42E05E
:1091A0000AC08DE10E941F58892B11F040E007C0D2
:1091B0008DE1602F44E0212F0E947048482F80915C
:1091C0006F0C90E08F709070242F30E0892B39F471
:1091D0002F703070232B71F0842F806406C02F70A5
:1091E0003070232B39F4842F806240936F0C1F91D1
:1091F0000F910895842FF9CF8BE00E941F5840E013
:109200002091C10230E08217930709F041E0440F3A
:10921000440F80914F0C8B7F842B80934F0C0895CB
:10922000EF92FF920F931F938C014AE3E42E4CE0E0
:10923000F42E6AE070E00E94865CC7014AE050E0CC
:109240000E94BC59C8016AE070E00E94865CBC01C3
:10925000C7014AE050E00E94BC591F910F91FF9056
:10926000EF900895CF93DF93EC0104C08AE39CE074
:109270000E94FC58FE01219664916623B9F7DF91A4
:10928000CF9108950F931F93CF93DF938C01462FB7
:109290008AE39CE060E00E94B441E80104C08AE3F4
:1092A0009CE00E94FC589E01201B822FFE0121960B
:1092B00064916623A1F7992787FD9095C0E1D0E0DE
:1092C000C81BD90B05C080E990E10E943249219763
:1092D000D7FFF9CFDF91CF911F910F910895EF92B2
:1092E000FF920F931F93CF93DF937C018C01F3E0E8
:1092F000000F111FFA95E1F7081B190B095D1D4FAF
:10930000F8018281938160E00E94424989E690E100
:1093100061E00E9442498AE39CE060E041E00E94F3
:10932000B441F801868180FF05C08AE39CE00E9479
:10933000984104C08AE39CE00E94A241F3E1EF1649
:10934000F10409F45EC084E1E816F10454F4E1E0AC
:10935000EE16F104B1F0FCE0EF16F10409F08CC058
:1093600065C08BE1E816F10409F46AC0ECE1EE1681
:10937000F10409F475C0F4E1EF16F10409F07CC0C2
:1093800047C080912E02C82FD0E0E097D7FD05C0DE
:1093900087E690E10E94324907C085E690E10E948D
:1093A0003249D095C195DF4FCE0164E070E00E9454
:1093B000865C8AE39CE04AE050E00E94BC5983E668
:1093C00090E10E943249CE0164E070E00E94865C28
:1093D000BC01E4E0660F771FEA95E1F7681B790BA3
:1093E00029F480E690E10E94324906C08AE39CE0BD
:1093F0004AE050E00E94BC598BE590E10E9432495E
:1094000061C089E590E10E9432496091AC0220C0C0
:109410008091B3028C3320F087E590E10E943249BD
:109420006091B30270E06C53704007C0709182028B
:1094300060E080917B02680F711D8AE39CE00BC0A5
:109440006091E4028DE070E00E9472586091E40245
:109450008AE39CE070E04AE050E00E94BC5932C0D0
:109460008091EB026FEF70E0681B71098CE00E9445
:1094700072586091EB02ECCFF70153E0EE0FFF1F43
:109480005A95E1F7EE19FF09E95DFD4F8181608191
:10949000813051F4662319F480E590E102C083E540
:1094A00090E10E94324907C08AE39CE070E04AE004
:1094B00050E00E94BC5987E1E816F10419F48EE4EB
:1094C00090E111C0C7014397029720F0E8E1EE1642
:1094D000F10419F489E490E106C0F1E1EF16F1041A
:1094E00021F484E490E10E943249DF91CF911F91F1
:1094F0000F91FF90EF900895EF92FF920F931F93BB
:10950000182F092F0E946F49212F302FC9018C017C
:109510008AEAE82E82E00E94B348482F282F30E0E4
:10952000C9018F70907082309105D9F08430910517
:1095300061F1019709F068C0F801B3E0EE0FFF1F79
:10954000BA95E1F7E01BF10BE95DFD4F868180FFE5
:109550005EC090818181891709F459C09F5F908313
:1095600056C0F801A3E0EE0FFF1FAA95E1F7E01B3C
:10957000F10BE95DFD4F868180FF46C08081882325
:1095800009F442C0815080833FC046FF3DC047FF81
:109590000BC080911503882311F0E09215030E94FF
:1095A000FD47FF24F39434C00330110541F480914A
:1095B0003C02882309F1FF240CE010E029C00C30A4
:1095C000110521F4FF240EE010E022C00531110541
:1095D00041F48091BA02882379F4FF2407E110E076
:1095E00017C00231110541F48091A502882321F4AE
:1095F000FF2405E110E00CC0C801019663E270E0B1
:109600000E94865C8C0103C0442309F483CFFF24AD
:10961000C8010E946F49FF2009F47CCF8AE39CE0D7
:109620000E94A2411F910F91FF90EF9008950F9318
:109630001F93CF93DF93482F062F8AE39CE060E0CF
:109640000E94B4418091500C8F7019F48FE790E123
:1096500010C08DE790E10E9432496091500C6F700C
:109660008AE39CE070E04AE050E00E94BC598BE73E
:1096700090E10E94324980914F0C80FD06C08FE638
:1096800090E161E00E94424926C0E091500CEF70E9
:10969000F0E0ED5AF34F1081C1E0D0E08091500C22
:1096A0008F7051F48091A50290E0C817D90721F47A
:1096B00010FD06C06DE405C010FD02C06FE501C0DD
:1096C000602F8AE39CE00E94FC582196C930D105A6
:1096D00011F01695E3CF8AE690E10E9432498AE3C1
:1096E0009CE06DE041E00E94B44180914F0C81FD0F
:1096F00006C082FF09C08091BA02882329F08AE35C
:109700009CE063E00E9466418AE39CE06EE041E0F9
:109710000E94B44180914F0C86FF05C08AE39CE013
:1097200062E00E9466418AE39CE06FE041E00E94B3
:10973000B44160E08091500C82958F7090E0039767
:109740000CF061E08AE39CE00E946641DF91CF91DA
:109750001F910F910895EF92FF920F931F93CF9354
:10976000DF938C017B018AE39CE00E94E3418AE362
:109770009CE060E040E00E94B441C0E0D0E0F8012D
:10978000EC0FFD1F60818AE39CE070E04AE050E04E
:109790000E94BC5985E890E10E9432492196C3306D
:1097A000D10569F7F80163818AE39CE070E04AE043
:1097B00050E00E94BC598AE39CE060E041E00E94D6
:1097C000B44183E890E10E9432498AE39CE0B7010A
:1097D0004AE050E00E94BC59DF91CF911F910F9158
:1097E000FF90EF90089520914F0C2170F999FECFD2
:1097F0001FBA80E390E092BD81BD20BD0FB6F89402
:10980000FA9AF99A0FBE20914F0C22952170F9997E
:10981000FECF1FBA81E390E092BD81BD20BD0FB69F
:10982000F894FA9AF99A0FBE4091650C5091660C23
:109830006091670C7091680C82E390E02DE137E451
:109840000E94BF090895F999FECF80E390E092BD90
:1098500081BDF89A90B5917080914F0C8E7F892BC5
:1098600080934F0CF999FECF81E390E092BD81BDCA
:10987000F89A90B591709295907F80914F0C8F7E61
:10988000892B80934F0C82E390E065E177E40E949E
:109890007D096093650C7093660C8093670C9093C0
:1098A000680C0895EF92FF920F931F93CF93DF936D
:1098B00083E060E00E94CB5708E51CE080914F0CEC
:1098C00080FD02C060E002C0F8016081C7E0D0E026
:1098D000E62EFF2486E160E00E94CB57B7010C2EF4
:1098E00002C0759567950A94E2F7617085E10E9460
:1098F000CB5786E161E00E94CB572197FFEFCF3F26
:10990000DF0741F7015010408CE002351807B1F62F
:1099100083E061E00E94CB57DF91CF911F910F91BF
:10992000FF90EF90089580914F0C8D7F80934F0CA6
:109930001092650C1092660C1092670C1092680CD5
:109940000E94F34B0E94524C089580914F0C82600C
:1099500080934F0C0E94F34B0E94524C08958091CB
:109960004F0C8E7F80934F0C0E94524C0E94F34B01
:10997000089580914F0C816080934F0C0E94524C4F
:109980000E94F34B0895AF92BF92CF92DF92FF9265
:109990000F931F93CF93DF935B016C01FF24C1E012
:1099A000D0E03CC08AE39CE00E94E3418AE39CE073
:1099B00060E040E00E94B4410F2D10E0B8016F5FFD
:1099C0007F4F8AE39CE04AE050E00E94BC5910922D
:1099D000530C1092540C1092550C1092560C10927D
:1099E000570C1092580C93E0169507959A95E1F74D
:1099F0000D5A134F8F2D87709E0102C0220F331F07
:109A00008A95E2F7C901F8012081282B20830E9462
:109A1000524CC601B5010E94D756F3948091520C66
:109A2000F81608F4BFCFFF24FBCF64EF71E080E0AD
:109A300090E00E94D756F999FECF12BC11BCF89A5B
:109A400090B5943620F48AE0989F902D11249D3C87
:109A500059F4F999FECF82E290E092BD81BDF89A67
:109A600080B58A3A09F091C00E94FD470E94F34BED
:109A700080E490E067E671E00E94214880E690E093
:109A800060E771E00E94214880E890E06AE771E0B9
:109A90000E94214882ED90E160E00E94424983ECFF
:109AA00090E161E00E94424980E091E0F999FECFA7
:109AB0001FBA92BD81BD10BC0FB6F894FA9AF99AFC
:109AC0000FBE019628E08030920781F720E031E058
:109AD000E1E0F0E043E5F999FECF1FBA32BD21BDC8
:109AE00040BD0FB6F894FA9AF99A0FBEF999FECFD5
:109AF0001FBA2F5F3F4F32BD21BD21503040CF01F3
:109B00006AE070E00E94865C605D60BD0FB6F8940C
:109B1000FA9AF99A0FBEF999FECF1FBA2E5F3F4FFE
:109B200032BD21BDCF016AE070E00E94865C805D9D
:109B300080BD0FB6F894FA9AF99A0FBE225F3F4F94
:109B400084E02030380711F03196C5CF80E694E0EC
:109B50002FEFF999FECF1FBA92BD81BD20BD0FB680
:109B6000F894FA9AF99A0FBE019634E08636930774
:109B700081F764EF71E080E090E00E94D756E091B9
:109B80006D0CF0916E0C099528C00E94DE4720E60E
:109B900034E0F999FECF32BD21BDF89A80B5F901C4
:109BA000E750F84F80832F5F3F4F84E02636380719
:109BB00081F726E634E0F999FECF32BD21BDF89A4F
:109BC00080B5F901E750F84F80832F5F3F4F84E065
:109BD0002C36380781F70E94234C80E00E94B3485E
:109BE00090E08F7090708230910521F18430910562
:109BF00021F1019709F04CC064E670E080E090E04C
:109C00000E94D7568DE10E941F58892B29F460E2EB
:109C100073E080E090E00BC06091CF0270E080E0E4
:109C200090E028EE33E040E050E00E94475C0E9464
:109C3000C34C2EC082E290E020C083EB90E160E054
:109C40000E94424960ED77E080E090E00E94D756A4
:109C500082EA90E160E00E94424982E990E161E09D
:109C60000E94424980E00E94B34886FFFBCF8AE30E
:109C70009CE00E94E34180E090E00E947C4A809159
:109C80001503882329F0E0916D0CF0916E0C099575
:109C90008CE061E00E948C578DE061E00E948C575F
:109CA0006091E4028DE070E00E9472588091EB02B6
:109CB0006FEF70E0681B71098CE00E947258089584
:109CC000DF93CF93CDB7DEB727970FB6F894DEBFFB
:109CD0000FBECDBFCE0101960E9451468C8190E00F
:109CE000059667E070E00E94865C27960FB6F894B0
:109CF000DEBF0FBECDBFCF91DF910895DF92EF920F
:109D0000FF920F931F93D82E0E94FD447B018C017C
:109D10008AE39CE060E04D2D0E94B441C801B70188
:109D20000E94EA430E9410498EE890E10E94324965
:109D3000C801B7010E94E4430E9410498BE890E1FA
:109D40000E9432490E94604EE82FF0E0EE0FFF1FA4
:109D5000E45EFC4F808191810E94324989E890E164
:109D60000E943249C801B7010E94D2430E941049A3
:109D700087E890E10E943249C801B7010E94DE43A2
:109D80000E9410491F910F91FF90EF90DF9008956E
:109D90008F92AF92CF92EF920F931F93DF93CF9357
:109DA000CDB7DEB768970FB6F894DEBF0FBECDBF54
:109DB00083E061E00E948C5781E061E00E948C5753
:109DC00086E161E00E948C5785E161E00E948C573A
:109DD00083E061E00E94CB5781E061E00E94CB57B5
:109DE0001092530C1092540C1092550C1092560C69
:109DF0001092570C1092580C0E94524C81E060E077
:109E00000E94CB5780E061E00E948C5780E061E0C7
:109E10000E94CB5781EC99E060E00E94AD3911E0DF
:109E2000109381008CE061E00E948C578DE061E02E
:109E30000E948C576091E4028DE070E00E9472589D
:109E40008091EB026FEF70E0681B71098CE00E945B
:109E5000725800D000D0EDB7FEB73196ADB7BEB79F
:109E600011961C921182128213828AE39CE061E0B7
:109E700043E12FEF02E1E4E1EE2E75E1C72E56E15A
:109E8000A52E37E1832E0E945A420F900F900F901B
:109E90000F908AE39CE060E142E020E00E94EB4109
:109EA0008BE060E00E948C578BE061E00E94CB5712
:109EB00085EC9CE00E940E5480914F0C816081786B
:109EC00080934F0C1092500C1093510C88E08093AB
:109ED000520C1092650C1092660C1092670C109246
:109EE000680C1092690C10926A0C10926B0C109214
:109EF0006C0CDE011196E6E7F3E001900D928150C3
:109F0000E1F7DE011996EEE6F3E088E001900D92AC
:109F10008150E1F7DE015196E6E6F3E088E001903A
:109F20000D928150E1F78AE39CE061E08E010F5FC2
:109F30001F4FA8010E9470411A821B8281E08C830E
:109F40008AE39CE060E0A8010E9470418AE39CE003
:109F500062E0AE01475F5F4F0E9470418AE39CE080
:109F600063E0AE014F5E5F4F0E9470418CE161E0A3
:109F70000E948C578CE160E00E94CB578FE160E03B
:109F80000E948C578EE160E00E948C578DE160E06A
:109F90000E948C578FE161E00E94CB578EE161E017
:109FA0000E94CB578DE161E00E94CB570E941E4674
:109FB000882329F480914F0C806280934F0C68961F
:109FC0000FB6F894DEBF0FBECDBFCF91DF911F91CA
:109FD0000F91EF90CF90AF908F9008950F931F93B4
:109FE000DF93CF93CDB7DEB728970FB6F894DEBFD7
:109FF0000FBECDBFFC018B018091DD02858384E81B
:10A0000093E0BF0144E00E94A635882311F490E05C
:10A0100032C0109305020093040280913C02882311
:10A0200019F00E94223921C08091430289838091D6
:10A030004A028A83809151028B83809158028C83DB
:10A0400080915F028D83809166028E8380916D0284
:10A050008F83809174028887CE010196BE016B5F69
:10A060007F4F40E050E00E94833590E0882309F460
:10A0700091E081E09827892F28960FB6F894DEBFEB
:10A080000FBECDBFCF91DF911F910F910895CF9358
:10A09000DF93DC01EB01722F632F822F932F9C0142
:10A0A000F90150E016C08081981771F431968081D3
:10A0B000882371F411968C918D3331F4872F962F6C
:10A0C0009C01F90151E004C0872F962F9C01F901F2
:10A0D00011969C91992339F0903229F09A3019F019
:10A0E000552309F304C0513011F030E018C06A2F35
:10A0F00050E04150504002C0299311963A2F361B30
:10A100002C91222359F0203249F02A3039F026329E
:10A1100029F0832F90E08417950774F31882832F1A
:10A12000DF91CF910895CF93DF93FC01EC0137C00D
:10A130008B3211F480E231C0853279F5DF0111965E
:10A140009181392F30533A3070F0892F8156863003
:10A1500010F4375208C0892F8154863010F030E057
:10A1600002C0392F3753FD01319611962C91922F51
:10A1700090539A3070F0822F8156863010F49752A7
:10A1800008C0822F8154863010F090E002C0922FD8
:10A190009753832F8295807F892B89933196808175
:10A1A000882331F61882DF91CF910895DC01FB01FD
:10A1B00086E001900D928150E1F708959C01FB012A
:10A1C00080819181A281B381F90180839183A283EF
:10A1D000B38308958093700C08951F93CF93DF93FA
:10A1E0000E94C956EB011FEF09C00E94C9566C1BA3
:10A1F0007D0B6955724010F08FE00CC01EBD0DB490
:10A2000007FEFDCF8EB58F3F81F38E3F11F481E0C5
:10A210000DC08DE08093720CE091730CF091740C82
:10A2200080819091750C892B808380E0DF91CF91A4
:10A230001F910895FF920F931F93CF93DF938C018B
:10A240000E94C956EB01FF24FA94FEBC0DB407FE30
:10A25000FDCF8EB58F3F11F481E008C00E94C95632
:10A260006C1B7D0B6017710780F380E0DF91CF914D
:10A270001F910F91FF900895DF92EF92FF920F933D
:10A280001F93182FD42EE52EF62E072FE091730C76
:10A29000F091740C90818091750C80958923808356
:10A2A0008CE291E00E941A51812F80648EBD0DB422
:10A2B00007FEFDCF0EBD0DB407FEFDCFFEBC0DB4F5
:10A2C00007FEFDCFEEBC0DB407FEFDCFDEBC0DB426
:10A2D00007FEFDCF112311F485E905C0183011F4F4
:10A2E00087E801C08FEF8EBD0DB407FEFDCF90E073
:10A2F0002FEF2EBD0DB407FEFDCF8EB587FF02C038
:10A300009150B9F71F910F91FF90EF90DF90089552
:10A31000EF92FF920F931F93CF93DF93EC017A019B
:10A320008B018091710C833039F089E0EE0CFF1CB9
:10A33000001F111F8A95D1F781E1B801A7010E9482
:10A340003C518823C9F70E94ED50882319F41092DC
:10A35000720C1BC08FEF8EBD20E030E09FEF0DB47C
:10A3600007FEFDCF8EB5FE01E20FF31F80839EBD79
:10A370002F5F3F4F81E02F3F380789F70DB407FE6D
:10A38000FDCF8EB5C150DE4F8883E091730CF09104
:10A39000740C80819091750C892B808380E0DF9113
:10A3A000CF911F910F91FF90EF900895DF92EF9260
:10A3B000FF920F931F93D82E7A018B0187E340E021
:10A3C00050E060E070E00E943C518D2DB801A70183
:10A3D0000E943C511F910F91FF90EF90DF900895E4
:10A3E000EF92FF920F931F93CF93DF93082F0E945A
:10A3F000C956EB01E091700C8E2F90E0FC01EF5FED
:10A40000FE4EE491F0E0EE0FFF1FE351FF4E259169
:10A4100034913093740C2093730C8F5D9E4EFC012D
:10A4200074917093750CE0912C038E2F90E0FC01D9
:10A43000EF5FFE4EE491F0E0EE0FFF1FE351FF4EA1
:10A44000A591B491B093770CA093760C8F5D9E4E3E
:10A45000FC0164916093780CE0912B034E2F50E047
:10A46000FA01EF5FFE4EE491F0E0EE0FFF1FE351C3
:10A47000FF4E8591949190937A0C8093790C4F5D67
:10A480005E4EFA01849180937B0CE0912D034E2F58
:10A4900050E0FA01EF5FFE4EE4918E2F90E0880FBE
:10A4A000991F83519F4EFC01E590F490F0927D0C32
:10A4B000E0927C0C4F5D5E4EFA01949190937E0C7D
:10A4C000F9018081872B8083F7018081892B80832C
:10A4D0008C91862B8C938091700C61E00E948C573C
:10A4E00080912B0361E00E948C5780912D0361E0E5
:10A4F0000E948C5780912C0360E00E948C578091C1
:10A500002A0361E00E948C5780912A0361E00E9437
:10A51000CB57E091730CF091740C80819091750C85
:10A52000892B808383E58CBD8DB58E7F8DBD80E0CA
:10A530002FEF2EBD0DB407FEFDCF8F5F8A30C9F718
:10A54000808190959823908309C00E94C9566C1B06
:10A550007D0B615D774010F081E048C080E040E015
:10A5600050E060E070E00E943C51182F813069F7A4
:10A5700088E04AEA51E060E070E00E943C5182FFCE
:10A5800003C01093710C1BC080E02FEF2EBD0DB4E3
:10A5900007FEFDCF9EB58F5F8430C1F79A3A11F068
:10A5A00082E024C082E08093710C09C00E94C956E9
:10A5B0006C1B7D0B615D774010F088E017C089E26D
:10A5C00040E050E060E070E00E94D651882371F7CF
:10A5D0008091710C823071F58AE340E050E060E0D8
:10A5E00070E00E943C51882379F086E08093720CE1
:10A5F000E091730CF091740C80819091750C892B13
:10A6000080838091720C29C08FEF8EBD0DB407FE40
:10A61000FDCF8EB5807C803C19F483E08093710C73
:10A6200080E09FEF9EBD0DB407FEFDCF2EB58F5F7E
:10A630008330C1F7E091730CF091740C808190919C
:10A64000750C892B8083073028F086E18093720C8B
:10A6500080E003C000650CBD81E0DF91CF911F91C8
:10A660000F91FF90EF90089581E08093C40C609368
:10A67000A10C1092C20C1092C30C08952091A00C52
:10A6800030E080919F0C281B3109C9010895409149
:10A690009F0C8091A00C481718F02FEF3FEF0AC0D5
:10A6A000E42FF0E0E158F34F8081282F30E04F5F36
:10A6B00040939F0CC9010895E0919F0C8091A00CDC
:10A6C000E81718F0EFEFFFEF06C0F0E0E158F34FA6
:10A6D0008081E82FF0E0CF01089508951092C80C12
:10A6E0001092C70C88EE93E0A0E0B0E08093C90C14
:10A6F0009093CA0CA093CB0CB093CC0C82E893E05F
:10A700009093C60C8093C50C0895CF92DF92EF9280
:10A71000FF920F931F93CF93DF937C016B018A010C
:10A720008091C40C8823A1F0C0E0D0E00DC0D70117
:10A73000ED91FC91D601AC0FBD1F0190F081E02D91
:10A74000C7016C9109952196C017D10780F304C009
:10A75000CB01642F0E94B754C801DF91CF911F91A4
:10A760000F91FF90EF90DF90CF900895DF93CF93FC
:10A770000F92CDB7DEB7FC0169838091C40C8823AA
:10A78000C9F08091C30C803238F081E090E093836F
:10A79000828320E030E015C08091C20CE82FF0E009
:10A7A000EE55F34F998190838F5F8093C20C809315
:10A7B000C30C05C0CE01019661E00E94B75421E0B0
:10A7C00030E0C9010F90CF91DF9108950F93062FCC
:10A7D0008091A10C62EA7CE04091C30C21E00E94D0
:10A7E00062541092C20C1092C30C1092C40C0F91C0
:10A7F000089561E00E94E6530895413208F040E276
:10A80000862F6FE77CE00E94195410929F0C809372
:10A81000A00C089521E00E94FD53089510929F0C12
:10A820001092A00C1092C20C1092C30C0E9463569E
:10A830000895382F413210F040E042C08091D10C91
:10A840008823E1F791E09093D10C2093D30C8FEF04
:10A8500080933E0D1092F90C41504093FA0C4F5FDB
:10A860009093D20C8091D20C330F832B8093D20C17
:10A870008091D40C813041F41092D40C8091D20C90
:10A880008093BB0085EC01C085EE8093BC00809175
:10A89000D10C8130E1F38091F90C841710F44091D0
:10A8A000F90C20E030E00AC0FB01E20FF31FD901F0
:10A8B000A752B34F8C9180832F5F3F4F2417A0F393
:10A8C000842F08950F931F93582F122F413210F0A9
:10A8D00081E04AC08091D10C8823E1F782E0809327
:10A8E000D10C0093D30C8FEF80933E0D1092F90C96
:10A8F0004093FA0CA9EDBCE0FB0102C081918D935D
:10A900008E2F861B8417D0F31092D20C8091D20C1C
:10A91000550F852B8093D20C8091D40C813041F45B
:10A920001092D40C8091D20C8093BB0085EC01C0B6
:10A9300085EE8093BC00112321F08091D10C8230F0
:10A94000E1F380913E0D8F3F11F480E00DC08091C6
:10A950003E0D803211F482E007C080913E0D8033BD
:10A9600011F084E001C083E01F910F910895482FFA
:10A97000613210F081E008958091D10C843011F0A3
:10A9800082E0089560931C0DABEFBCE0842F9C0126
:10A99000F90102C081918D938E2F841B8617D0F30D
:10A9A00080E008951F920F920FB60F9211242F93FB
:10A9B0003F934F935F936F937F938F939F93AF9347
:10A9C000BF93EF93FF938091B90090E0887F9070E0
:10A9D0008036910509F4F2C081369105CCF58832B4
:10A9E000910509F47BC089329105B4F48031910559
:10A9F00009F46FC0813191053CF4009709F447C117
:10AA0000089709F04FC165C08831910509F466C007
:10AA1000809709F047C182C08034910509F4A4C031
:10AA20008134910544F48033910509F482C0C897BC
:10AA300009F038C189C08035910509F489C088358D
:10AA4000910509F496C08834910509F02BC1AEC078
:10AA50008839910509F413C189399105ECF48837D7
:10AA6000910509F4ABC0893791054CF488369105FE
:10AA700009F4A4C08037910509F014C19FC088383B
:10AA8000910509F4FCC08039910509F49DC0803816
:10AA9000910509F007C198C0803B910509F4C6C033
:10AAA000813B91054CF4803A910509F49FC0883AA6
:10AAB000910509F0F7C0BAC0803C910509F4E3C0E4
:10AAC000883C910509F4DFC0883B910509F0EAC094
:10AAD000C2C08091D20C8093BB00CFC09091F90C82
:10AAE0008091FA0C981768F49091F90CE92FF0E036
:10AAF000E752F34F80818093BB009F5F9093F90CE6
:10AB0000BCC08091D30C882309F44BC085ED8093A1
:10AB1000BC008091BC0084FDFCCFC2C080E2809369
:10AB20003E0D85ED8093BC008091BC0084FDFCCF80
:10AB3000B7C080E380933E0D85ED8093BC0080918B
:10AB4000BC0084FDFCCFACC088E380933E0D9BC06D
:10AB50008091F90C9091BB00E82FF0E0E752F34FA1
:10AB600090838F5F8093F90C9091F90C8091FA0C8F
:10AB700082C08091F90C9091BB00E82FF0E0E75281
:10AB8000F34F90838F5F8093F90C8091D30C8823CF
:10AB900041F085ED8093BC008091BC0084FDFCCF2A
:10ABA0007FC081E08093D40C84EA6EC085ED8093F1
:10ABB000BC008091BC0084FDFCCF72C083E0809318
:10ABC000D10C10923D0D59C080913D0D803208F09E
:10ABD00056C080913D0D9091BB00E82FF0E0E35E00
:10ABE000F24F90838F5F80933D0D47C080913D0D64
:10ABF000803230F4E0913D0DF0E0E35EF24F1082E0
:10AC000085ED8093BC008091BC0084FDFCCF109248
:10AC1000D10C60913D0DE091D70CF091D80C8DE1F5
:10AC20009DE070E0099510923D0D2DC084E0809369
:10AC3000D10C10921B0D10921C0DE091D50CF091CF
:10AC4000D60C099580911C0D882329F481E080930E
:10AC50001C0D1092FB0C90911B0DE92FF0E0E550BC
:10AC6000F34F80818093BB009F5F90931B0D909169
:10AC70001B0D80911C0D981710F485EC01C085E820
:10AC80008093BC000FC085EC8093BC0009C010927B
:10AC90003E0D85ED8093BC008091BC0084FDFCCF0F
:10ACA0001092D10CFF91EF91BF91AF919F918F9135
:10ACB0007F916F915F914F913F912F910F900FBEB8
:10ACC0000F901F9018951092D10C81E08093D30CB7
:10ACD0001092D40C81E161E00E94CB5780E161E0E9
:10ACE0000E94CB57E9EBF0E080818E7F80838081EA
:10ACF0008D7F808384E38093B80085E48093BC00DB
:10AD000008951F920F920FB60F9211242F933F9325
:10AD10008F939F93AF93BF938091430D9091440D78
:10AD2000A091450DB091460D3091470D0196A11DA2
:10AD3000B11D232F235D2D3720F02D570196A11D26
:10AD4000B11D2093470D8093430D9093440DA09324
:10AD5000450DB093460D80913F0D9091400DA0910F
:10AD6000410DB091420D0196A11DB11D80933F0D83
:10AD70009093400DA093410DB093420DBF91AF91C0
:10AD80009F918F913F912F910F900FBE0F901F9029
:10AD900018958FB7F8942091430D3091440D409150
:10ADA000450D5091460D8FBFB901CA010895EF922C
:10ADB000FF920F931F937B018C019FB7F894209112
:10ADC0003F0D3091400D4091410D5091420D86B59F
:10ADD000A89B06C08F3F21F02F5F3F4F4F4F5F4F23
:10ADE0009FBF542F432F322F2227280F311D411D83
:10ADF000511DDA01C90162E0880F991FAA1FBB1F0C
:10AE00006A95D1F7820F931FA41FB51FBC0135C0EF
:10AE10009FB7F89420913F0D3091400D4091410D26
:10AE20005091420D86B5A89B06C08F3F21F02F5F41
:10AE30003F4F4F4F5F4F9FBF542F432F322F22273B
:10AE4000280F311D411D511DDA01C901E2E0880FB3
:10AE5000991FAA1FBB1FEA95D1F7820F931FA41F4A
:10AE6000B51F861B970B885E934090F20894E1080B
:10AE7000F1080109110968517C4FE114F104010541
:10AE8000110531F61F910F91FF90EF9008950197F2
:10AE900039F0880F991F880F991F02970197F1F7D2
:10AEA0000895789484B5826084BD84B5816084BD42
:10AEB00085B5826085BD85B5816085BDEEE6F0E033
:10AEC000808181608083E1E8F0E01082808182608F
:10AED0008083808181608083E0E8F0E08081816010
:10AEE0008083E1EBF0E0808184608083E0EBF0E040
:10AEF000808181608083EAE7F0E0808184608083E4
:10AF0000808182608083808181608083808180688D
:10AF100080831092C1000895CF93DF93482F50E0B3
:10AF2000CA018F5D9E4EFC0134914F5F5E4EFA0167
:10AF30008491882369F190E0880F991FFC01ED51FD
:10AF4000FF4EA591B491FC01E351FF4EC591D49100
:10AF5000662351F42FB7F8948C91932F9095892301
:10AF60008C93888189230BC0623061F42FB7F894E9
:10AF70008C91932F909589238C938881832B888340
:10AF80002FBF06C09FB7F8948C91832B8C939FBFE3
:10AF9000DF91CF910895482F50E0CA018F5B9E4EFC
:10AFA000FC012491CA018F5D9E4EFC0194914F5F7C
:10AFB0005E4EFA013491332309F440C0222351F14B
:10AFC000233071F0243028F42130A1F0223011F523
:10AFD00014C02630B1F02730C1F02430D9F404C0B9
:10AFE000809180008F7703C0809180008F7D809357
:10AFF000800010C084B58F7702C084B58F7D84BD7A
:10B0000009C08091B0008F7703C08091B0008F7D20
:10B010008093B000E32FF0E0EE0FFF1FE351FF4EEF
:10B02000A591B4912FB7F894662321F48C91909553
:10B03000892302C08C91892B8C932FBF0895682F90
:10B0400070E0CB018F5B9E4EFC012491CB018F5DA4
:10B050009E4EFC0144916F5F7E4EFB0194919923BB
:10B0600019F420E030E03CC0222351F1233071F08C
:10B07000243028F42130A1F0223011F514C02630FC
:10B08000B1F02730C1F02430D9F404C080918000A1
:10B090008F7703C0809180008F7D8093800010C0E7
:10B0A00084B58F7702C084B58F7D84BD09C080913F
:10B0B000B0008F7703C08091B0008F7D8093B00087
:10B0C000892F90E0880F991F89509F4EFC01A59110
:10B0D000B4918C9120E030E0842311F021E030E045
:10B0E000C90108951F93CF93DF93182FEB0161E0FF
:10B0F0000E948C57209709F44AC0CF3FD10509F42C
:10B1000049C0E12FF0E0EF5BFE4E84918330C1F047
:10B11000843028F4813051F08230B1F50CC0863093
:10B1200019F1873049F1843079F514C084B580680D
:10B1300084BDC7BD33C084B5806284BDC8BD2EC088
:10B1400080918000806880938000D0938900C093B4
:10B15000880024C080918000806280938000D0931A
:10B160008B00C0938A001AC08091B00080688093E1
:10B17000B000C093B30012C08091B0008062809391
:10B18000B000C093B4000AC0C038D1051CF4812FB0
:10B1900060E002C0812F61E00E94CB57DF91CF9128
:10B1A0001F910895CF92DF92EF92FF920F931F931A
:10B1B000CF93DF937C016B018A01C0E0D0E00FC028
:10B1C000D6016D916D01D701ED91FC910190F08157
:10B1D000E02DC7010995C80FD91F01501040011576
:10B1E000110571F7CE01DF91CF911F910F91FF9063
:10B1F000EF90DF90CF900895DC01ED91FC910190EC
:10B20000F081E02D09950895CF93DF93DB010D9038
:10B210000020E9F71197A61BB70BEC01E881F98133
:10B220000280F381E02DAD010995DF91CF91089562
:10B230004F925F927F928F929F92AF92BF92CF92E6
:10B24000DF92EF92FF920F931F93DF93CF93CDB7CF
:10B25000DEB7A1970FB6F894DEBF0FBECDBF2C01AD
:10B26000742ECB01223008F42AE019A231E2C32E59
:10B27000D12CCC0EDD1E822E9924AA24BB24672D4E
:10B28000752FA50194010E94995C79018A01C8017A
:10B29000B701A50194010E94475C472D461B089405
:10B2A000C108D1084A3014F4405D01C0495CF60180
:10B2B0004083E114F1040105110521F07E2C5F2D7E
:10B2C000C801DDCFC201B6010E940459A1960FB694
:10B2D000F894DEBF0FBECDBFCF91DF911F910F91CC
:10B2E000FF90EF90DF90CF90BF90AF909F908F90A6
:10B2F0007F905F904F900895CF92DF92EF92FF92F0
:10B300000F931F93CF93DF93EC016A017B0121150B
:10B31000310541F4E881F9810190F081E02D642F3D
:10B3200009951FC02A303105D1F477FF17C0E88195
:10B33000F9810190F081E02D6DE209958C0144279F
:10B340005527BA014C195D096E097F09CE012AE023
:10B350000E9418599801280F391F04C02AE00E9442
:10B3600018599C01C901DF91CF911F910F91FF9056
:10B37000EF90DF90CF900895EF92FF920F931F937D
:10B380007B019A010027F7FC0095102FB801A70157
:10B390000E947C591F910F91FF90EF90089508959E
:10B3A0001F920F920FB60F9211242F933F934F933A
:10B3B0008F939F93EF93FF934091C6002091880D48
:10B3C0003091890D2F5F3F4F2F73307080918A0D20
:10B3D00090918B0D2817390759F0E091880DF09165
:10B3E000890DE85BF24F40833093890D2093880DDF
:10B3F000FF91EF919F918F914F913F912F910F90DE
:10B400000FBE0F901F901895E091DC0DF091DD0DAF
:10B41000E05CFF4F8191919120813181821B930BE0
:10B420008F739070892B11F00E94CF5908951F924D
:10B430000F920FB60F9211242F933F938F939F93E8
:10B44000EF93FF932091CC0D3091CD0D8091CE0DD7
:10B450009091CF0D2817390731F48091C1008F7D6D
:10B460008093C10014C0E091CE0DF091CF0DE45750
:10B47000F24F20818091CE0D9091CF0D01968F7368
:10B4800090709093CF0D8093CE0D2093C600FF91C6
:10B49000EF919F918F913F912F910F900FBE0F9041
:10B4A0001F901895DC011C96ED91FC911D97E05CB6
:10B4B000FF4F2191319180819181281B390B2F738E
:10B4C0003070C9010895DC011C96ED91FC911D9727
:10B4D000E05CFF4F20813181E054F040DF01AE5B42
:10B4E000BF4F8D919C9111972817390719F42FEFB1
:10B4F0003FEF07C08D919C91E80FF91F8081282FA5
:10B5000030E0C9010895DC011C96ED91FC911D9776
:10B51000E05CFF4F20813181E054F040DF01AE5B01
:10B52000BF4F8D919C9111972817390719F42FEF70
:10B530003FEF10C08D919C911197E80FF91F20816A
:10B540008D919C91119701968F73907011969C9399
:10B550008E9330E0C9010895FC0186859785DC0152
:10B56000A05CBF4FFC01EE5BFF4F2D913C9111970A
:10B570008081918128173907C1F70895CF93DF9310
:10B58000EC01EE85FF85E05CFF4F20813181E054C6
:10B59000F0402F5F3F4F2F733070DF01AE5BBF4F26
:10B5A0008D919C91119728173907D1F3E05CFF4FDB
:10B5B00080819181E054F040E80FF91F6083EE85AF
:10B5C000FF85E05CFF4F31832083EE89FF89208176
:10B5D00081E090E00D8C02C0880F991F0A94E2F779
:10B5E000282B208381E090E0DF91CF910895109285
:10B5F000D30D1092D20D88EE93E0A0E0B0E08093DE
:10B60000D40D9093D50DA093D60DB093D70D82E9AC
:10B6100093E09093D10D8093D00D88E49DE09093BA
:10B62000DD0D8093DC0D8CE89DE09093DF0D809321
:10B63000DE0D85EC90E09093E10D8093E00D84ECBD
:10B6400090E09093E30D8093E20D80EC90E0909376
:10B65000E50D8093E40D81EC90E09093E70D8093ED
:10B66000E60D86EC90E09093E90D8093E80D84E080
:10B670008093EA0D83E08093EB0D87E08093EC0DDF
:10B6800085E08093ED0D81E08093EE0D0895CF93DA
:10B69000DF930E9451570E940C29C4E0DAE50E9412
:10B6A000D7292097E1F30E94045AF9CFE89409C002
:10B6B00097FB3EF490958095709561957F4F8F4FE5
:10B6C0009F4F9923A9F0F92F96E9BB279395F695FB
:10B6D000879577956795B795F111F8CFFAF4BB0F79
:10B6E00011F460FF1BC06F5F7F4F8F4F9F4F16C0DD
:10B6F000882311F096E911C0772321F09EE8872F67
:10B70000762F05C0662371F096E8862F70E060E022
:10B710002AF09A95660F771F881FDAF7880F96959B
:10B72000879597F9089597F99F6780E870E060E042
:10B7300008959FEF80EC089500240A9416161706CA
:10B7400018060906089500240A9412161306140612
:10B7500005060895092E0394000C11F4882352F075
:10B76000BB0F40F4BF2B11F460FF04C06F5F7F4F2D
:10B770008F4F9F4F089557FD9058440F551F59F014
:10B780005F3F71F04795880F97FB991F61F09F3FCE
:10B7900079F087950895121613061406551FF2CFF7
:10B7A0004695F1DF08C0161617061806991FF1CF47
:10B7B00086957105610508940895E894BB2766276E
:10B7C0007727CB0197F908950BD0C4CFB5DF28F0C8
:10B7D000BADF18F0952309F0A6CFABCF1124EECF36
:10B7E000CADFA0F3959FD1F3950F50E0551F629FDC
:10B7F000F001729FBB27F00DB11D639FAA27F00DCA
:10B80000B11DAA1F649F6627B00DA11D661F829FF0
:10B810002227B00DA11D621F739FB00DA11D621FD5
:10B82000839FA00D611D221F749F3327A00D611DF2
:10B83000231F849F600D211D822F762F6A2F1124D4
:10B840009F5750408AF0E1F088234AF0EE0FFF1F27
:10B85000BB1F661F771F881F91505040A9F79E3F5E
:10B86000510570F060CFAACF5F3FECF3983EDCF358
:10B87000869577956795B795F795E7959F5FC1F79B
:10B88000FE2B880F911D9695879597F90895629FD5
:10B89000D001739FF001829FE00DF11D649FE00DC8
:10B8A000F11D929FF00D839FF00D749FF00D659F29
:10B8B000F00D9927729FB00DE11DF91F639FB00D28
:10B8C000E11DF91FBD01CF0111240895991B79E0F5
:10B8D00004C0991F961708F0961B881F7A95C9F720
:10B8E00080950895AA1BBB1B51E107C0AA1FBB1F6F
:10B8F000A617B70710F0A61BB70B881F991F5A95FC
:10B90000A9F780959095BC01CD01089597FB092E6C
:10B9100007260AD077FD04D0E5DF06D000201AF410
:10B92000709561957F4F0895F6F7909581959F4F9B
:10B930000895A1E21A2EAA1BBB1BFD010DC0AA1F70
:10B94000BB1FEE1FFF1FA217B307E407F50720F088
:10B95000A21BB30BE40BF50B661F771F881F991F03
:10B960001A9469F760957095809590959B01AC014C
:10B97000BD01CF010895EE0FFF1F0590F491E02D5A
:10B9800009942F923F924F925F926F927F928F9283
:10B990009F92AF92BF92CF92DF92EF92FF920F935E
:10B9A0001F93CF93DF93CDB7DEB7CA1BDB0B0FB668
:10B9B000F894DEBF0FBECDBF09942A883988488825
:10B9C0005F846E847D848C849B84AA84B984C884BB
:10B9D000DF80EE80FD800C811B81AA81B981CE0FB2
:10B9E000D11D0FB6F894DEBF0FBECDBFED01089597
:04B9F000F894FFCFF9
:10B9F400687474703A2F2F72617973686F62627918
:10BA04002E6E65742F736372697074732F6A617616
:10BA1400612F737663322E302E35007400707700F8
:10BA24006C6F6300747474006E70770063707700D9
:10BA34006A7370007069640064006D007900763D7B
:10BA44005B0072736E0072627400656E006D6D004F
:10BA5400726400743D5B006F70656E646F6F72009A
:10BA6400426F73746F6E2C4D4100687474703A2F7A
:10BA74002F72617973686F6262792E6E65742F73A9
:10BA84006372697074732F6A6176612F737663329F
:10BA94002E302E35000069692D31007BD1016625D9
:10BAA400D401BD22D701561DDA018123DD011824FA
:10BAB400E0012D21E301CE0EE601C119E901FA11DD
:10BAC400EF011417F201B51BF5012B16F8018326BB
:10BAD400FB01890CFE012C180102B21E0402B80FEE
:10BAE4000702D10B0A02C90D0D02531B1002300DBF
:10BAF4000100010A50004F70656E537072696E6BDD
:10BB04006C65722D3030003703010306FF638253E6
:10BB1400633501100E0000CD004A0EB50D00206CF7
:10BB2400580EB90D030101630EBC0D0301016D0E26
:10BB3400C00D01C0FF770EC50D01A8FF830EC90D0E
:10BB44000101FF8F0ECD0D0116FF9B0ED10D01C01B
:10BB5400FFA70ED50D01A8FFB40ED90D0101FFC139
:10BB64000EDD0D0101FFCE0EE10D0150FFDB0EE5F0
:10BB74000D0200FFE60EE90D020101E70EED0D03D3
:10BB84000005F70EF00D030101080FF40D0300F09A
:10BB9400190FF80D030008280FFC0D03003C380FA3
:10BBA400000E033C78490F050E0300015A0F0A0EDC
:10BBB4000301016B0F0E0E0364FA7A0F120E030ACF
:10BBC400F0880F150E010001970F190E0300FFA84E
:10BBD4000F1E0E036EFFB30F240E0164FFC10F2866
:10BBE4000E0105FFD00F2C0E01CCFFDD0F300E012E
:10BBF40009FFED0F350E0136FFFD0F3A0E0177FFF9
:10BC04000D103F0E0100011D10440E0128102C10D0
:10BC14003010341038103C104010040506070000A2
:10BC240000006D0AD2586F000000002E6F4FFFFF16
:10BC3400FFFFFFFFFFFFFFFFFFFF00000000664163
:10BC4400D25800004000140054001F1C1F1E1F1E69
:10BC54001F1F1E1F1E1F000006091F0015150000D0
:10BC64001F111F11131E00140815010505150000EE
:10BC74000000B65385533E5347535C536D53000045
:0EBC84000000BE5AD258525A835A635AAC5A24
:00000001FF
